 followref003

 Timestamp is c9d5419f (reproducible build file hash)

 Preferred load address is 0000000180000000

 Start         Length     Name                   Class
 0001:00000000 00005400H .text$mn                CODE
 0001:00005400 00000036H .text$mn$00             CODE
 0001:00005436 00000092H .text$x                 CODE
 0002:00000000 000001c8H .idata$5                DATA
 0002:000001c8 00000038H .00cfg                  DATA
 0002:00000200 00000008H .CRT$XCA                DATA
 0002:00000208 00000008H .CRT$XCZ                DATA
 0002:00000210 00000008H .CRT$XIA                DATA
 0002:00000218 00000008H .CRT$XIC                DATA
 0002:00000220 00000008H .CRT$XIZ                DATA
 0002:00000228 00000008H .CRT$XLA                DATA
 0002:00000230 00000008H .CRT$XLZ                DATA
 0002:00000238 00000008H .CRT$XPA                DATA
 0002:00000240 00000008H .CRT$XPZ                DATA
 0002:00000248 00000008H .CRT$XTA                DATA
 0002:00000250 00000010H .CRT$XTZ                DATA
 0002:00000258 00000000H .gehcont$y              DATA
 0002:00000258 00000000H .gfids$y                DATA
 0002:00000260 00003720H .rdata                  DATA
 0002:00003980 00000000H .rdata$CastGuardVftablesA DATA
 0002:00003980 00000000H .rdata$CastGuardVftablesC DATA
 0002:00003980 00000028H .rdata$T                DATA
 0002:000039a8 000000bcH .rdata$voltmd           DATA
 0002:00003a64 0000031cH .rdata$zzzdbg           DATA
 0002:00003d80 00000008H .rtc$IAA                DATA
 0002:00003d88 00000008H .rtc$IZZ                DATA
 0002:00003d90 00000008H .rtc$TAA                DATA
 0002:00003d98 00000008H .rtc$TZZ                DATA
 0002:00003da0 00000004H .tls                    DATA
 0002:00003da4 00000004H .tls$                   DATA
 0002:00003da8 00000008H .tls$ZZZ                DATA
 0002:00003db0 00000400H .xdata                  DATA
 0002:000041b0 00000364H .edata                  DATA
 0002:00004514 0000008cH .idata$2                DATA
 0002:000045a0 00000018H .idata$3                DATA
 0002:000045b8 000001c8H .idata$4                DATA
 0002:00004780 00000486H .idata$6                DATA
 0003:00000000 00000190H .data                   DATA
 0003:00000190 00021758H .bss                    DATA
 0004:00000000 00000468H .pdata                  DATA

  Address         Publics by Value              Rva+Base               Lib:Object

 0000:00000000       __AbsoluteZero             0000000000000000     <absolute>
 0000:00000000       ___safe_se_handler_count   0000000000000000     <absolute>
 0000:00000000       ___safe_se_handler_table   0000000000000000     <absolute>
 0000:00000000       __arm64x_extra_rfe_table   0000000000000000     <absolute>
 0000:00000000       __arm64x_extra_rfe_table_size 0000000000000000     <absolute>
 0000:00000000       __arm64x_native_entrypoint 0000000000000000     <absolute>
 0000:00000000       __arm64x_redirection_metadata 0000000000000000     <absolute>
 0000:00000000       __arm64x_redirection_metadata_count 0000000000000000     <absolute>
 0000:00000000       __dynamic_value_reloc_table 0000000000000000     <absolute>
 0000:00000000       __enclave_config           0000000000000000     <absolute>
 0000:00000000       __guard_check_icall_a64n_fptr 0000000000000000     <absolute>
 0000:00000000       __guard_eh_cont_count      0000000000000000     <absolute>
 0000:00000000       __guard_eh_cont_table      0000000000000000     <absolute>
 0000:00000000       __guard_fids_count         0000000000000000     <absolute>
 0000:00000000       __guard_fids_table         0000000000000000     <absolute>
 0000:00000000       __guard_iat_count          0000000000000000     <absolute>
 0000:00000000       __guard_iat_table          0000000000000000     <absolute>
 0000:00000000       __guard_longjmp_count      0000000000000000     <absolute>
 0000:00000000       __guard_longjmp_table      0000000000000000     <absolute>
 0000:00000000       __hybrid_auxiliary_iat     0000000000000000     <absolute>
 0000:00000000       __hybrid_auxiliary_iat_copy 0000000000000000     <absolute>
 0000:00000000       __hybrid_code_map          0000000000000000     <absolute>
 0000:00000000       __hybrid_code_map_count    0000000000000000     <absolute>
 0000:00000000       __x64_code_ranges_to_entry_points 0000000000000000     <absolute>
 0000:00000000       __x64_code_ranges_to_entry_points_count 0000000000000000     <absolute>
 0000:00000100       __guard_flags              0000000000000100     <absolute>
 0000:00000000       __ImageBase                0000000180000000     <linker-defined>
 0001:00000000       ?NewObject@JNIEnv_@@QEAAPEAV_jobject@@PEAV_jclass@@PEAU_jmethodID@@ZZ 0000000180001000 f i libfollowref003.obj
 0001:00000028       ?TranslateError@@YAPEBDW4jvmtiError@@@Z 0000000180001028 f   libfollowref003.obj
 0001:000002e0       ?nsk_jni_check_exception@@YAHPEAUJNIEnv_@@QEBDH@Z 00000001800012e0 f   libfollowref003.obj
 0001:00000424       ?nsk_jni_lverify@@YAHHPEAUJNIEnv_@@HQEBDH1ZZ 0000000180001424 f   libfollowref003.obj
 0001:000004c4       Agent_Initialize           00000001800014c4 f   libfollowref003.obj
 0001:00000838       Agent_OnAttach             0000000180001838 f   libfollowref003.obj
 0001:00000838       Agent_OnLoad               0000000180001838 f   libfollowref003.obj
 0001:00000840       Java_nsk_jvmti_unit_FollowReferences_FollowRefObjects_addRefToVerify 0000000180001840 f   libfollowref003.obj
 0001:00000a18       Java_nsk_jvmti_unit_FollowReferences_FollowRefObjects_getTag 0000000180001a18 f   libfollowref003.obj
 0001:00000ad8       Java_nsk_jvmti_unit_FollowReferences_FollowRefObjects_resetRefsToVerify 0000000180001ad8 f   libfollowref003.obj
 0001:00000ae0       Java_nsk_jvmti_unit_FollowReferences_FollowRefObjects_resetTags 0000000180001ae0 f   libfollowref003.obj
 0001:00000b24       Java_nsk_jvmti_unit_FollowReferences_FollowRefObjects_setTag 0000000180001b24 f   libfollowref003.obj
 0001:00000d7c       Java_nsk_share_jvmti_ArgumentHandler_getAgentOptionsString 0000000180001d7c f   libfollowref003.obj
 0001:00000e2c       Java_nsk_share_jvmti_DebugeeClass_checkStatus 0000000180001e2c f   libfollowref003.obj
 0001:00000eb4       Java_nsk_share_jvmti_DebugeeClass_resetAgentData 0000000180001eb4 f   libfollowref003.obj
 0001:00000f14       Java_nsk_share_jvmti_RedefineAgent_agentStatus 0000000180001f14 f   libfollowref003.obj
 0001:00000f20       Java_nsk_share_jvmti_RedefineAgent_isRedefined 0000000180001f20 f   libfollowref003.obj
 0001:00000f2c       Java_nsk_share_jvmti_RedefineAgent_redefineAttempted 0000000180001f2c f   libfollowref003.obj
 0001:00000f38       MA_checkStatus             0000000180001f38 f   libfollowref003.obj
 0001:00000fdc       __local_stdio_printf_options 0000000180001fdc f i libfollowref003.obj
 0001:000016bc       arrayPrimitiveValueCallback 00000001800026bc f   libfollowref003.obj
 0001:00001a54       exitOnError                0000000180002a54 f   libfollowref003.obj
 0001:00001b08       fprintf                    0000000180002b08 f i libfollowref003.obj
 0001:00002810       heapReferenceCallback      0000000180003810 f   libfollowref003.obj
 0001:00002dd8       nsk_complain               0000000180003dd8 f   libfollowref003.obj
 0001:00002e04       nsk_jvmti_createJVMTIEnv   0000000180003e04 f   libfollowref003.obj
 0001:00002f34       nsk_jvmti_findOptionIntValue 0000000180003f34 f   libfollowref003.obj
 0001:00002fd0       nsk_jvmti_findOptionValue  0000000180003fd0 f   libfollowref003.obj
 0001:00003048       nsk_jvmti_lverify          0000000180004048 f   libfollowref003.obj
 0001:00003138       nsk_jvmti_parseOptions     0000000180004138 f   libfollowref003.obj
 0001:00003388       nsk_jvmti_resetAgentData   0000000180004388 f   libfollowref003.obj
 0001:00003408       nsk_jvmti_resumeSync       0000000180004408 f   libfollowref003.obj
 0001:000034b0       nsk_jvmti_setFailStatus    00000001800044b0 f   libfollowref003.obj
 0001:000034ec       nsk_jvmti_waitForSync      00000001800044ec f   libfollowref003.obj
 0001:000035f0       nsk_lcomplain              00000001800045f0 f   libfollowref003.obj
 0001:00003610       nsk_ldisplay               0000000180004610 f   libfollowref003.obj
 0001:00003630       nsk_ltrace                 0000000180004630 f   libfollowref003.obj
 0001:00003650       nsk_lvcomplain             0000000180004650 f   libfollowref003.obj
 0001:00003808       nsk_lvdisplay              0000000180004808 f   libfollowref003.obj
 0001:00003854       nsk_lverify                0000000180004854 f   libfollowref003.obj
 0001:000038b0       nsk_lvtrace                00000001800048b0 f   libfollowref003.obj
 0001:00003910       nsk_printf                 0000000180004910 f   libfollowref003.obj
 0001:00003938       nsk_vprintf                0000000180004938 f   libfollowref003.obj
 0001:000039ec       primitiveFieldCallback     00000001800049ec f   libfollowref003.obj
 0001:00003a30       printf                     0000000180004a30 f i libfollowref003.obj
 0001:00004308       stringPrimitiveValueCallback 0000000180005308 f   libfollowref003.obj
 0001:000044d4       __raise_securityfailure    00000001800054d4 f   MSVCRT:gs_report.obj
 0001:00004508       __report_gsfailure         0000000180005508 f   MSVCRT:gs_report.obj
 0001:00004748       __GSHandlerCheck           0000000180005748 f   MSVCRT:gshandler.obj
 0001:00004768       __GSHandlerCheckCommon     0000000180005768 f   MSVCRT:gshandler.obj
 0001:000047e0       __security_check_cookie    00000001800057e0 f   MSVCRT:amdsecgs.obj
 0001:00004b20       _DllMainCRTStartup         0000000180005b20 f   MSVCRT:dll_dllmain.obj
 0001:00004b60       __scrt_acquire_startup_lock 0000000180005b60 f   MSVCRT:utility.obj
 0001:00004b9c       __scrt_dllmain_after_initialize_c 0000000180005b9c f   MSVCRT:utility.obj
 0001:00004bd0       __scrt_dllmain_before_initialize_c 0000000180005bd0 f   MSVCRT:utility.obj
 0001:00004be8       __scrt_dllmain_crt_thread_attach 0000000180005be8 f   MSVCRT:utility.obj
 0001:00004c10       __scrt_dllmain_crt_thread_detach 0000000180005c10 f   MSVCRT:utility.obj
 0001:00004c28       __scrt_dllmain_exception_filter 0000000180005c28 f   MSVCRT:utility.obj
 0001:00004c88       __scrt_dllmain_uninitialize_c 0000000180005c88 f   MSVCRT:utility.obj
 0001:00004cb8       __scrt_dllmain_uninitialize_critical 0000000180005cb8 f   MSVCRT:utility.obj
 0001:00004ccc       __scrt_initialize_crt      0000000180005ccc f   MSVCRT:utility.obj
 0001:00004d18       __scrt_initialize_onexit_tables 0000000180005d18 f   MSVCRT:utility.obj
 0001:00004da4       __scrt_is_nonwritable_in_current_image 0000000180005da4 f   MSVCRT:utility.obj
 0001:00004e3c       __scrt_release_startup_lock 0000000180005e3c f   MSVCRT:utility.obj
 0001:00004e60       __scrt_uninitialize_crt    0000000180005e60 f   MSVCRT:utility.obj
 0001:00004e8c       _onexit                    0000000180005e8c f   MSVCRT:utility.obj
 0001:00004ec8       atexit                     0000000180005ec8 f   MSVCRT:utility.obj
 0001:00004ee0       __crt_debugger_hook        0000000180005ee0 f   MSVCRT:utility_desktop.obj
 0001:00004ee8       __scrt_fastfail            0000000180005ee8 f   MSVCRT:utility_desktop.obj
 0001:00005034       _guard_check_icall_nop     0000000180006034 f i MSVCRT:guard_support.obj
 0001:00005038       __security_init_cookie     0000000180006038 f   MSVCRT:gs_support.obj
 0001:000050e4       DllMain                    00000001800060e4 f   MSVCRT:dll_dllmain_stub.obj
 0001:00005108       ?__scrt_initialize_type_info@@YAXXZ 0000000180006108 f   MSVCRT:tncleanup.obj
 0001:00005118       ?__scrt_uninitialize_type_info@@YAXXZ 0000000180006118 f   MSVCRT:tncleanup.obj
 0001:00005124       __local_stdio_scanf_options 0000000180006124 f i MSVCRT:default_local_stdio_options.obj
 0001:0000512c       __scrt_initialize_default_local_stdio_options 000000018000612c f   MSVCRT:default_local_stdio_options.obj
 0001:00005148       __scrt_get_dyn_tls_init_callback 0000000180006148 f   MSVCRT:dyn_tls_init.obj
 0001:00005150       _RTC_Initialize            0000000180006150 f   MSVCRT:initsect.obj
 0001:0000518c       _RTC_Terminate             000000018000618c f   MSVCRT:initsect.obj
 0001:000051c8       __isa_available_init       00000001800061c8 f   MSVCRT:cpu_disp.obj
 0001:00005374       _get_startup_argv_mode     0000000180006374 f   MSVCRT:argv_mode.obj
 0001:0000537c       __scrt_is_ucrt_dll_in_use  000000018000637c f   MSVCRT:ucrt_detection.obj
 0001:00005390       memcpy                     0000000180006390 f   vcruntime:VCRUNTIME140.dll
 0001:00005396       memset                     0000000180006396 f   vcruntime:VCRUNTIME140.dll
 0001:0000539c       strchr                     000000018000639c f   vcruntime:VCRUNTIME140.dll
 0001:000053a2       __C_specific_handler       00000001800063a2 f   vcruntime:VCRUNTIME140.dll
 0001:000053a8       __std_type_info_destroy_list 00000001800063a8 f   vcruntime:VCRUNTIME140.dll
 0001:000053ae       strcmp                     00000001800063ae f   ucrt:api-ms-win-crt-string-l1-1-0.dll
 0001:000053b4       strlen                     00000001800063b4 f   ucrt:api-ms-win-crt-string-l1-1-0.dll
 0001:000053ba       _initterm                  00000001800063ba f   ucrt:api-ms-win-crt-runtime-l1-1-0.dll
 0001:000053c0       _initterm_e                00000001800063c0 f   ucrt:api-ms-win-crt-runtime-l1-1-0.dll
 0001:000053c6       _seh_filter_dll            00000001800063c6 f   ucrt:api-ms-win-crt-runtime-l1-1-0.dll
 0001:000053cc       _configure_narrow_argv     00000001800063cc f   ucrt:api-ms-win-crt-runtime-l1-1-0.dll
 0001:000053d2       _initialize_narrow_environment 00000001800063d2 f   ucrt:api-ms-win-crt-runtime-l1-1-0.dll
 0001:000053d8       _initialize_onexit_table   00000001800063d8 f   ucrt:api-ms-win-crt-runtime-l1-1-0.dll
 0001:000053de       _register_onexit_function  00000001800063de f   ucrt:api-ms-win-crt-runtime-l1-1-0.dll
 0001:000053e4       _execute_onexit_table      00000001800063e4 f   ucrt:api-ms-win-crt-runtime-l1-1-0.dll
 0001:000053ea       _crt_atexit                00000001800063ea f   ucrt:api-ms-win-crt-runtime-l1-1-0.dll
 0001:000053f0       _cexit                     00000001800063f0 f   ucrt:api-ms-win-crt-runtime-l1-1-0.dll
 0001:000053f8       __acrt_initialize          00000001800063f8 f   MSVCRT:ucrt_stubs.obj
 0001:000053f8       __acrt_thread_attach       00000001800063f8 f   MSVCRT:ucrt_stubs.obj
 0001:000053f8       __acrt_thread_detach       00000001800063f8 f   MSVCRT:ucrt_stubs.obj
 0001:000053f8       __acrt_uninitialize        00000001800063f8 f   MSVCRT:ucrt_stubs.obj
 0001:000053f8       __acrt_uninitialize_critical 00000001800063f8 f   MSVCRT:ucrt_stubs.obj
 0001:000053f8       __scrt_stub_for_acrt_initialize 00000001800063f8 f   MSVCRT:ucrt_stubs.obj
 0001:000053f8       __scrt_stub_for_acrt_thread_attach 00000001800063f8 f   MSVCRT:ucrt_stubs.obj
 0001:000053f8       __scrt_stub_for_acrt_thread_detach 00000001800063f8 f   MSVCRT:ucrt_stubs.obj
 0001:000053f8       __scrt_stub_for_acrt_uninitialize 00000001800063f8 f   MSVCRT:ucrt_stubs.obj
 0001:000053f8       __scrt_stub_for_acrt_uninitialize_critical 00000001800063f8 f   MSVCRT:ucrt_stubs.obj
 0001:000053f8       __vcrt_initialize          00000001800063f8 f   MSVCRT:ucrt_stubs.obj
 0001:000053f8       __vcrt_thread_attach       00000001800063f8 f   MSVCRT:ucrt_stubs.obj
 0001:000053f8       __vcrt_thread_detach       00000001800063f8 f   MSVCRT:ucrt_stubs.obj
 0001:000053f8       __vcrt_uninitialize        00000001800063f8 f   MSVCRT:ucrt_stubs.obj
 0001:000053f8       __vcrt_uninitialize_critical 00000001800063f8 f   MSVCRT:ucrt_stubs.obj
 0001:000053fc       __scrt_stub_for_is_c_termination_complete 00000001800063fc f   MSVCRT:ucrt_stubs.obj
 0001:000053fc       _is_c_termination_complete 00000001800063fc f   MSVCRT:ucrt_stubs.obj
 0001:00005410       _guard_dispatch_icall_nop  0000000180006410 f   MSVCRT:guard_dispatch.obj
 0001:00005430       _guard_xfg_dispatch_icall_nop 0000000180006430 f   MSVCRT:guard_xfg_dispatch.obj
 0002:00000000       __imp_RtlCaptureContext    0000000180007000     kernel32:KERNEL32.dll
 0002:00000008       __imp_RtlLookupFunctionEntry 0000000180007008     kernel32:KERNEL32.dll
 0002:00000010       __imp_RtlVirtualUnwind     0000000180007010     kernel32:KERNEL32.dll
 0002:00000018       __imp_UnhandledExceptionFilter 0000000180007018     kernel32:KERNEL32.dll
 0002:00000020       __imp_SetUnhandledExceptionFilter 0000000180007020     kernel32:KERNEL32.dll
 0002:00000028       __imp_GetCurrentProcess    0000000180007028     kernel32:KERNEL32.dll
 0002:00000030       __imp_TerminateProcess     0000000180007030     kernel32:KERNEL32.dll
 0002:00000038       __imp_IsProcessorFeaturePresent 0000000180007038     kernel32:KERNEL32.dll
 0002:00000040       __imp_CloseHandle          0000000180007040     kernel32:KERNEL32.dll
 0002:00000048       __imp_InitializeCriticalSectionAndSpinCount 0000000180007048     kernel32:KERNEL32.dll
 0002:00000050       __imp_DeleteCriticalSection 0000000180007050     kernel32:KERNEL32.dll
 0002:00000058       __imp_CreateEventW         0000000180007058     kernel32:KERNEL32.dll
 0002:00000060       __imp_GetModuleHandleW     0000000180007060     kernel32:KERNEL32.dll
 0002:00000068       __imp_GetProcAddress       0000000180007068     kernel32:KERNEL32.dll
 0002:00000070       __imp_IsDebuggerPresent    0000000180007070     kernel32:KERNEL32.dll
 0002:00000078       __imp_QueryPerformanceCounter 0000000180007078     kernel32:KERNEL32.dll
 0002:00000080       __imp_GetCurrentProcessId  0000000180007080     kernel32:KERNEL32.dll
 0002:00000088       __imp_GetCurrentThreadId   0000000180007088     kernel32:KERNEL32.dll
 0002:00000090       __imp_GetSystemTimeAsFileTime 0000000180007090     kernel32:KERNEL32.dll
 0002:00000098       __imp_DisableThreadLibraryCalls 0000000180007098     kernel32:KERNEL32.dll
 0002:000000a0       __imp_InitializeSListHead  00000001800070a0     kernel32:KERNEL32.dll
 0002:000000a8       \177KERNEL32_NULL_THUNK_DATA 00000001800070a8     kernel32:KERNEL32.dll
 0002:000000b0       __imp_memcpy               00000001800070b0     vcruntime:VCRUNTIME140.dll
 0002:000000b8       __imp_memset               00000001800070b8     vcruntime:VCRUNTIME140.dll
 0002:000000c0       __imp_strchr               00000001800070c0     vcruntime:VCRUNTIME140.dll
 0002:000000c8       __imp___C_specific_handler 00000001800070c8     vcruntime:VCRUNTIME140.dll
 0002:000000d0       __imp___std_type_info_destroy_list 00000001800070d0     vcruntime:VCRUNTIME140.dll
 0002:000000d8       \177VCRUNTIME140_NULL_THUNK_DATA 00000001800070d8     vcruntime:VCRUNTIME140.dll
 0002:000000e0       __imp_strtol               00000001800070e0     ucrt:api-ms-win-crt-convert-l1-1-0.dll
 0002:000000e8       \177api-ms-win-crt-convert-l1-1-0_NULL_THUNK_DATA 00000001800070e8     ucrt:api-ms-win-crt-convert-l1-1-0.dll
 0002:000000f0       __imp_malloc               00000001800070f0     ucrt:api-ms-win-crt-heap-l1-1-0.dll
 0002:000000f8       __imp_free                 00000001800070f8     ucrt:api-ms-win-crt-heap-l1-1-0.dll
 0002:00000100       \177api-ms-win-crt-heap-l1-1-0_NULL_THUNK_DATA 0000000180007100     ucrt:api-ms-win-crt-heap-l1-1-0.dll
 0002:00000108       __imp__errno               0000000180007108     ucrt:api-ms-win-crt-runtime-l1-1-0.dll
 0002:00000110       __imp_exit                 0000000180007110     ucrt:api-ms-win-crt-runtime-l1-1-0.dll
 0002:00000118       __imp__cexit               0000000180007118     ucrt:api-ms-win-crt-runtime-l1-1-0.dll
 0002:00000120       __imp__crt_atexit          0000000180007120     ucrt:api-ms-win-crt-runtime-l1-1-0.dll
 0002:00000128       __imp__execute_onexit_table 0000000180007128     ucrt:api-ms-win-crt-runtime-l1-1-0.dll
 0002:00000130       __imp__register_onexit_function 0000000180007130     ucrt:api-ms-win-crt-runtime-l1-1-0.dll
 0002:00000138       __imp__initialize_onexit_table 0000000180007138     ucrt:api-ms-win-crt-runtime-l1-1-0.dll
 0002:00000140       __imp__initialize_narrow_environment 0000000180007140     ucrt:api-ms-win-crt-runtime-l1-1-0.dll
 0002:00000148       __imp__configure_narrow_argv 0000000180007148     ucrt:api-ms-win-crt-runtime-l1-1-0.dll
 0002:00000150       __imp__seh_filter_dll      0000000180007150     ucrt:api-ms-win-crt-runtime-l1-1-0.dll
 0002:00000158       __imp__initterm_e          0000000180007158     ucrt:api-ms-win-crt-runtime-l1-1-0.dll
 0002:00000160       __imp__initterm            0000000180007160     ucrt:api-ms-win-crt-runtime-l1-1-0.dll
 0002:00000168       \177api-ms-win-crt-runtime-l1-1-0_NULL_THUNK_DATA 0000000180007168     ucrt:api-ms-win-crt-runtime-l1-1-0.dll
 0002:00000170       __imp___acrt_iob_func      0000000180007170     ucrt:api-ms-win-crt-stdio-l1-1-0.dll
 0002:00000178       __imp_fflush               0000000180007178     ucrt:api-ms-win-crt-stdio-l1-1-0.dll
 0002:00000180       __imp___stdio_common_vsprintf 0000000180007180     ucrt:api-ms-win-crt-stdio-l1-1-0.dll
 0002:00000188       __imp___stdio_common_vfprintf 0000000180007188     ucrt:api-ms-win-crt-stdio-l1-1-0.dll
 0002:00000190       \177api-ms-win-crt-stdio-l1-1-0_NULL_THUNK_DATA 0000000180007190     ucrt:api-ms-win-crt-stdio-l1-1-0.dll
 0002:00000198       __imp_strcmp               0000000180007198     ucrt:api-ms-win-crt-string-l1-1-0.dll
 0002:000001a0       __imp__strdup              00000001800071a0     ucrt:api-ms-win-crt-string-l1-1-0.dll
 0002:000001a0       __imp_strdup               00000001800071a0     ucrt:api-ms-win-crt-string-l1-1-0.dll
 0002:000001a8       __imp_strlen               00000001800071a8     ucrt:api-ms-win-crt-string-l1-1-0.dll
 0002:000001b0       __imp_strpbrk              00000001800071b0     ucrt:api-ms-win-crt-string-l1-1-0.dll
 0002:000001b8       __imp_strncpy              00000001800071b8     ucrt:api-ms-win-crt-string-l1-1-0.dll
 0002:000001c0       \177api-ms-win-crt-string-l1-1-0_NULL_THUNK_DATA 00000001800071c0     ucrt:api-ms-win-crt-string-l1-1-0.dll
 0002:000001c8       __guard_check_icall_fptr   00000001800071c8     MSVCRT:guard_support.obj
 0002:000001d0       __guard_xfg_check_icall_fptr 00000001800071d0     MSVCRT:guard_support.obj
 0002:000001d8       __guard_dispatch_icall_fptr 00000001800071d8     MSVCRT:guard_support.obj
 0002:000001e0       __guard_xfg_dispatch_icall_fptr 00000001800071e0     MSVCRT:guard_support.obj
 0002:000001e8       __guard_xfg_table_dispatch_icall_fptr 00000001800071e8     MSVCRT:guard_support.obj
 0002:000001f0       __castguard_check_failure_os_handled_fptr 00000001800071f0     MSVCRT:guard_support.obj
 0002:000001f8       __guard_memcpy_fptr        00000001800071f8     vcruntime:softmemtag.obj
 0002:00000200       __xc_a                     0000000180007200     MSVCRT:initializers.obj
 0002:00000208       __xc_z                     0000000180007208     MSVCRT:initializers.obj
 0002:00000210       __xi_a                     0000000180007210     MSVCRT:initializers.obj
 0002:00000220       __xi_z                     0000000180007220     MSVCRT:initializers.obj
 0002:00000228       __xl_a                     0000000180007228     MSVCRT:tlssup.obj
 0002:00000230       __xl_z                     0000000180007230     MSVCRT:tlssup.obj
 0002:00000238       __xp_a                     0000000180007238     MSVCRT:initializers.obj
 0002:00000240       __xp_z                     0000000180007240     MSVCRT:initializers.obj
 0002:00000248       __xt_a                     0000000180007248     MSVCRT:initializers.obj
 0002:00000250       __xt_z                     0000000180007250     MSVCRT:initializers.obj
 0002:00000260       g_refKindStr               0000000180007260     libfollowref003.obj
 0002:00000410       ??_C@_09BPLDFGCI@unknown_0@ 0000000180007410     libfollowref003.obj
 0002:00000420       ??_C@_0BL@FPNMECJD@JVMTI_HEAP_REFERENCE_CLASS@ 0000000180007420     libfollowref003.obj
 0002:00000440       ??_C@_0BL@FKGKKLNM@JVMTI_HEAP_REFERENCE_FIELD@ 0000000180007440     libfollowref003.obj
 0002:00000460       ??_C@_0CD@CAEHCFJF@JVMTI_HEAP_REFERENCE_ARRAY_ELEM@ 0000000180007460     libfollowref003.obj
 0002:00000488       ??_C@_0CC@DNEBMCNK@JVMTI_HEAP_REFERENCE_CLASS_LOAD@ 0000000180007488     libfollowref003.obj
 0002:000004b0       ??_C@_0BN@CJMIPEBB@JVMTI_HEAP_REFERENCE_SIGNERS@ 00000001800074b0     libfollowref003.obj
 0002:000004d0       ??_C@_0CH@HBOIDPEB@JVMTI_HEAP_REFERENCE_PROTECTION@ 00000001800074d0     libfollowref003.obj
 0002:000004f8       ??_C@_0BP@MDKGDGKL@JVMTI_HEAP_REFERENCE_INTERFACE@ 00000001800074f8     libfollowref003.obj
 0002:00000518       ??_C@_0CC@JJMIHNJH@JVMTI_HEAP_REFERENCE_STATIC_FIE@ 0000000180007518     libfollowref003.obj
 0002:00000540       ??_C@_0CD@IDHEEGID@JVMTI_HEAP_REFERENCE_CONSTANT_P@ 0000000180007540     libfollowref003.obj
 0002:00000568       ??_C@_0CA@EFFCHNG@JVMTI_HEAP_REFERENCE_SUPERCLASS@ 0000000180007568     libfollowref003.obj
 0002:00000588       ??_C@_0L@PCDFHGCJ@unknown_11@ 0000000180007588     libfollowref003.obj
 0002:00000598       ??_C@_0L@NJBICFOK@unknown_12@ 0000000180007598     libfollowref003.obj
 0002:000005a8       ??_C@_0L@MAADBEKL@unknown_13@ 00000001800075a8     libfollowref003.obj
 0002:000005b8       ??_C@_0L@IPECICGM@unknown_14@ 00000001800075b8     libfollowref003.obj
 0002:000005c8       ??_C@_0L@JGFJLDCN@unknown_15@ 00000001800075c8     libfollowref003.obj
 0002:000005d8       ??_C@_0L@LNHEOAOO@unknown_16@ 00000001800075d8     libfollowref003.obj
 0002:000005e8       ??_C@_0L@KEGPNBKP@unknown_17@ 00000001800075e8     libfollowref003.obj
 0002:000005f8       ??_C@_0L@CDPHMNGA@unknown_18@ 00000001800075f8     libfollowref003.obj
 0002:00000608       ??_C@_0L@DKOMPMCB@unknown_19@ 0000000180007608     libfollowref003.obj
 0002:00000618       ??_C@_0L@OJGIPJDB@unknown_20@ 0000000180007618     libfollowref003.obj
 0002:00000628       ??_C@_0CA@KAOFNDEM@JVMTI_HEAP_REFERENCE_JNI_GLOBAL@ 0000000180007628     libfollowref003.obj
 0002:00000648       ??_C@_0CC@HPFAJBK@JVMTI_HEAP_REFERENCE_SYSTEM_CLA@ 0000000180007648     libfollowref003.obj
 0002:00000670       ??_C@_0BN@FDEGFOHC@JVMTI_HEAP_REFERENCE_MONITOR@ 0000000180007670     libfollowref003.obj
 0002:00000690       ??_C@_0CB@HKIBCMAJ@JVMTI_HEAP_REFERENCE_STACK_LOCA@ 0000000180007690     libfollowref003.obj
 0002:000006b8       ??_C@_0BP@EAACMMOE@JVMTI_HEAP_REFERENCE_JNI_LOCAL@ 00000001800076b8     libfollowref003.obj
 0002:000006d8       ??_C@_0BM@IJDEOGOE@JVMTI_HEAP_REFERENCE_THREAD@ 00000001800076d8     libfollowref003.obj
 0002:000006f8       ??_C@_0BL@EDGPPKC@JVMTI_HEAP_REFERENCE_OTHER@ 00000001800076f8     libfollowref003.obj
 0002:00000714       ??_C@_04BCJPDBDA@Code@     0000000180007714     libfollowref003.obj
 0002:00000720       ??_C@_0BA@OCLMCFKC@LineNumberTable@ 0000000180007720     libfollowref003.obj
 0002:00000730       ??_C@_0BD@CPAEPILC@LocalVariableTable@ 0000000180007730     libfollowref003.obj
 0002:00000748       ??_C@_0BH@NMBDNHBD@LocalVariableTypeTable@ 0000000180007748     libfollowref003.obj
 0002:00000760       ??_C@_0O@HIHEEDNJ@StackMapTable@ 0000000180007760     libfollowref003.obj
 0002:00000770       ??_C@_0BA@NAMAECDA@REFERENCE_CLASS@ 0000000180007770     libfollowref003.obj
 0002:00000780       ??_C@_0BA@NFHGKLHP@REFERENCE_FIELD@ 0000000180007780     libfollowref003.obj
 0002:00000790       ??_C@_0BI@EDCHCAFJ@REFERENCE_ARRAY_ELEMENT@ 0000000180007790     libfollowref003.obj
 0002:000007a8       ??_C@_0BH@FLCINHMH@REFERENCE_CLASS_LOADER@ 00000001800077a8     libfollowref003.obj
 0002:000007c0       ??_C@_0BC@KMOCJECH@REFERENCE_SIGNERS@ 00000001800077c0     libfollowref003.obj
 0002:000007d8       ??_C@_0BM@PKPOPHFB@REFERENCE_PROTECTION_DOMAIN@ 00000001800077d8     libfollowref003.obj
 0002:000007f8       ??_C@_0BE@HAIEDKM@REFERENCE_INTERFACE@ 00000001800077f8     libfollowref003.obj
 0002:00000810       ??_C@_0BH@PPKBGIIK@REFERENCE_STATIC_FIELD@ 0000000180007810     libfollowref003.obj
 0002:00000828       ??_C@_0BI@OABEEDEP@REFERENCE_CONSTANT_POOL@ 0000000180007828     libfollowref003.obj
 0002:00000840       ??_C@_0L@OLCOEHGI@unknown_10@ 0000000180007840     libfollowref003.obj
 0002:00000850       ??_C@_0BF@DOEFOIJK@REFERENCE_JNI_GLOBAL@ 0000000180007850     libfollowref003.obj
 0002:00000868       ??_C@_0BH@GBJMBMAH@REFERENCE_SYSTEM_CLASS@ 0000000180007868     libfollowref003.obj
 0002:00000880       ??_C@_0BC@NGGMDOEE@REFERENCE_MONITOR@ 0000000180007880     libfollowref003.obj
 0002:00000898       ??_C@_0BG@BFKPPLND@REFERENCE_STACK_LOCAL@ 0000000180007898     libfollowref003.obj
 0002:000008b0       ??_C@_0BE@IEKMLJOD@REFERENCE_JNI_LOCAL@ 00000001800078b0     libfollowref003.obj
 0002:000008c8       ??_C@_0BB@MGGEAILG@REFERENCE_THREAD@ 00000001800078c8     libfollowref003.obj
 0002:000008e0       ??_C@_0BA@ILCKPPAB@REFERENCE_OTHER@ 00000001800078e0     libfollowref003.obj
 0002:000008f0       ??_C@_0L@HCDIAMJG@?9?5?$CFs?0?5?$CFd?3?5@ 00000001800078f0     libfollowref003.obj
 0002:00000900       ??_C@_0JI@HLPECLFI@?$CD?5?4?4?4?6?$CD?5ERROR?3?5too?5many?5complai@ 0000000180007900     libfollowref003.obj
 0002:000009a0       ??_C@_0ED@JNEKCCOB@The?5following?5fake?5exception?5st@ 00000001800079a0     libfollowref003.obj
 0002:000009e8       ??_C@_0CN@FCNMDFBH@nsk?4share?4Fake_Exception_for_RU@ 00000001800079e8     libfollowref003.obj
 0002:00000a18       ??_C@_08PGFFNAEI@?$CI?$CFs?3?$CFd?$CJ?5@ 0000000180007a18     libfollowref003.obj
 0002:00000a28       ??_C@_0DP@IENMAEGI@s?2test?2hotspot?2jtreg?2vmTestbase@ 0000000180007a28     libfollowref003.obj
 0002:00000a68       ??_C@_0BL@NDJLFFJB@?7at?5nsk_lvcomplain?$CI?$CFs?3?$CFd?$CJ?6@ 0000000180007a68     libfollowref003.obj
 0002:00000a88       ??_C@_0BC@JOOKAFKF@?$CD?5ERROR?3?5?$CFs?0?5?$CFd?3?5@ 0000000180007a88     libfollowref003.obj
 0002:00000aa0       ??_C@_09KJEAHMEH@?$CD?5ERROR?3?5@ 0000000180007aa0     libfollowref003.obj
 0002:00000aac       ??_C@_02GPIOPFAK@?$DO?$DO@ 0000000180007aac     libfollowref003.obj
 0002:00000ab0       ??_C@_02FODMEDOG@?$DM?$DM@ 0000000180007ab0     libfollowref003.obj
 0002:00000ab4       ??_C@_02DJGKEECL@?4?4@     0000000180007ab4     libfollowref003.obj
 0002:00000ab8       ??_C@_0O@CJPGJOAF@?9?5?$CFs?0?5?$CFd?3?5?$CFs?5@ 0000000180007ab8     libfollowref003.obj
 0002:00000ac8       ??_C@_0CB@IAKPDOIC@?$CD?5?5?5verified?5assertion?5is?5FALSE@ 0000000180007ac8     libfollowref003.obj
 0002:00000af0       ??_C@_0CO@LGONDEPD@stdout?3?5fflush?5failed?5?9?5err?$DN?$CFd?5@ 0000000180007af0     libfollowref003.obj
 0002:00000b20       ??_C@_0CO@KBGKJPBD@stderr?3?5fflush?5failed?5?9?5err?$DN?$CFd?5@ 0000000180007b20     libfollowref003.obj
 0002:00000b50       ??_C@_0BB@JCNMKLLK@JVMTI_ERROR_NONE@ 0000000180007b50     libfollowref003.obj
 0002:00000b68       ??_C@_0BL@LDIMKLPH@JVMTI_ERROR_INVALID_THREAD@ 0000000180007b68     libfollowref003.obj
 0002:00000b88       ??_C@_0CB@PJFPAIKJ@JVMTI_ERROR_INVALID_THREAD_GROU@ 0000000180007b88     libfollowref003.obj
 0002:00000bb0       ??_C@_0BN@LLMKHMNF@JVMTI_ERROR_INVALID_PRIORITY@ 0000000180007bb0     libfollowref003.obj
 0002:00000bd0       ??_C@_0CB@MBOFKAGB@JVMTI_ERROR_THREAD_NOT_SUSPENDE@ 0000000180007bd0     libfollowref003.obj
 0002:00000bf8       ??_C@_0BN@FABOLPBI@JVMTI_ERROR_THREAD_SUSPENDED@ 0000000180007bf8     libfollowref003.obj
 0002:00000c18       ??_C@_0BN@FDGNOBJM@JVMTI_ERROR_THREAD_NOT_ALIVE@ 0000000180007c18     libfollowref003.obj
 0002:00000c38       ??_C@_0BL@GOBIFKNJ@JVMTI_ERROR_INVALID_OBJECT@ 0000000180007c38     libfollowref003.obj
 0002:00000c58       ??_C@_0BK@FCMAJPPC@JVMTI_ERROR_INVALID_CLASS@ 0000000180007c58     libfollowref003.obj
 0002:00000c78       ??_C@_0BP@IKLLBKEB@JVMTI_ERROR_CLASS_NOT_PREPARED@ 0000000180007c78     libfollowref003.obj
 0002:00000c98       ??_C@_0BN@KLPPLKG@JVMTI_ERROR_INVALID_METHODID@ 0000000180007c98     libfollowref003.obj
 0002:00000cb8       ??_C@_0BN@BCEKOKND@JVMTI_ERROR_INVALID_LOCATION@ 0000000180007cb8     libfollowref003.obj
 0002:00000cd8       ??_C@_0BM@DFDGPME@JVMTI_ERROR_INVALID_FIELDID@ 0000000180007cd8     libfollowref003.obj
 0002:00000cf8       ??_C@_0BL@NELIEPEC@JVMTI_ERROR_NO_MORE_FRAMES@ 0000000180007cf8     libfollowref003.obj
 0002:00000d18       ??_C@_0BJ@BDBECFDM@JVMTI_ERROR_OPAQUE_FRAME@ 0000000180007d18     libfollowref003.obj
 0002:00000d38       ??_C@_0BK@MIIFNLOB@JVMTI_ERROR_TYPE_MISMATCH@ 0000000180007d38     libfollowref003.obj
 0002:00000d58       ??_C@_0BJ@HPCAOILC@JVMTI_ERROR_INVALID_SLOT@ 0000000180007d58     libfollowref003.obj
 0002:00000d78       ??_C@_0BG@CHILOPNI@JVMTI_ERROR_DUPLICATE@ 0000000180007d78     libfollowref003.obj
 0002:00000d90       ??_C@_0BG@DIEMLHKM@JVMTI_ERROR_NOT_FOUND@ 0000000180007d90     libfollowref003.obj
 0002:00000da8       ??_C@_0BM@NHMCKHOB@JVMTI_ERROR_INVALID_MONITOR@ 0000000180007da8     libfollowref003.obj
 0002:00000dc8       ??_C@_0BO@PPEDAJGL@JVMTI_ERROR_NOT_MONITOR_OWNER@ 0000000180007dc8     libfollowref003.obj
 0002:00000de8       ??_C@_0BG@FCAIPEID@JVMTI_ERROR_INTERRUPT@ 0000000180007de8     libfollowref003.obj
 0002:00000e00       ??_C@_0CB@EGDBNKOI@JVMTI_ERROR_INVALID_CLASS_FORMA@ 0000000180007e00     libfollowref003.obj
 0002:00000e28       ??_C@_0CG@DGKOGIAL@JVMTI_ERROR_CIRCULAR_CLASS_DEFI@ 0000000180007e28     libfollowref003.obj
 0002:00000e50       ??_C@_0BP@ICEALPKC@JVMTI_ERROR_FAILS_VERIFICATION@ 0000000180007e50     libfollowref003.obj
 0002:00000e70       ??_C@_0DC@JDACLMIO@JVMTI_ERROR_UNSUPPORTED_REDEFIN@ 0000000180007e70     libfollowref003.obj
 0002:00000ea8       ??_C@_0DE@GKDKNOMJ@JVMTI_ERROR_UNSUPPORTED_REDEFIN@ 0000000180007ea8     libfollowref003.obj
 0002:00000ee0       ??_C@_0BO@LAFKIOG@JVMTI_ERROR_INVALID_TYPESTATE@ 0000000180007ee0     libfollowref003.obj
 0002:00000f00       ??_C@_0DH@INDGCLLB@JVMTI_ERROR_UNSUPPORTED_REDEFIN@ 0000000180007f00     libfollowref003.obj
 0002:00000f38       ??_C@_0DE@NHEOMMGI@JVMTI_ERROR_UNSUPPORTED_REDEFIN@ 0000000180007f38     libfollowref003.obj
 0002:00000f70       ??_C@_0CA@EKPNJOEP@JVMTI_ERROR_UNSUPPORTED_VERSION@ 0000000180007f70     libfollowref003.obj
 0002:00000f90       ??_C@_0BN@OFFMAHHL@JVMTI_ERROR_NAMES_DONT_MATCH@ 0000000180007f90     libfollowref003.obj
 0002:00000fb0       ??_C@_0DN@HHBBLAKE@JVMTI_ERROR_UNSUPPORTED_REDEFIN@ 0000000180007fb0     libfollowref003.obj
 0002:00000ff0       ??_C@_0DO@HMBGBGNA@JVMTI_ERROR_UNSUPPORTED_REDEFIN@ 0000000180007ff0     libfollowref003.obj
 0002:00001030       ??_C@_0BP@PBECGKHJ@JVMTI_ERROR_UNMODIFIABLE_CLASS@ 0000000180008030     libfollowref003.obj
 0002:00001050       ??_C@_0BK@CANILEHF@JVMTI_ERROR_NOT_AVAILABLE@ 0000000180008050     libfollowref003.obj
 0002:00001070       ??_C@_0CE@INJKMEFK@JVMTI_ERROR_MUST_POSSESS_CAPABI@ 0000000180008070     libfollowref003.obj
 0002:00001098       ??_C@_0BJ@LBFPFPDM@JVMTI_ERROR_NULL_POINTER@ 0000000180008098     libfollowref003.obj
 0002:000010b8       ??_C@_0BP@CHJPNNEM@JVMTI_ERROR_ABSENT_INFORMATION@ 00000001800080b8     libfollowref003.obj
 0002:000010d8       ??_C@_0BP@OMFMNLC@JVMTI_ERROR_INVALID_EVENT_TYPE@ 00000001800080d8     libfollowref003.obj
 0002:000010f8       ??_C@_0BN@BIBNPHHO@JVMTI_ERROR_ILLEGAL_ARGUMENT@ 00000001800080f8     libfollowref003.obj
 0002:00001118       ??_C@_0BK@KKNDHDCE@JVMTI_ERROR_NATIVE_METHOD@ 0000000180008118     libfollowref003.obj
 0002:00001138       ??_C@_0BK@PMKCFHAE@JVMTI_ERROR_OUT_OF_MEMORY@ 0000000180008138     libfollowref003.obj
 0002:00001158       ??_C@_0BK@NNJBDMNB@JVMTI_ERROR_ACCESS_DENIED@ 0000000180008158     libfollowref003.obj
 0002:00001178       ??_C@_0BI@GHECLMNC@JVMTI_ERROR_WRONG_PHASE@ 0000000180008178     libfollowref003.obj
 0002:00001190       ??_C@_0BF@OLIHJOII@JVMTI_ERROR_INTERNAL@ 0000000180008190     libfollowref003.obj
 0002:000011a8       ??_C@_0BO@EOHGKJHI@JVMTI_ERROR_UNATTACHED_THREAD@ 00000001800081a8     libfollowref003.obj
 0002:000011c8       ??_C@_0CA@LKHFDACL@JVMTI_ERROR_INVALID_ENVIRONMENT@ 00000001800081c8     libfollowref003.obj
 0002:000011e8       ??_C@_0BA@MMFHLOKK@?$DMunknown?5error?$DO@ 00000001800081e8     libfollowref003.obj
 0002:000011f8       ??_C@_0CF@CBHOKDB@throwable?5?$DN?5jni?9?$DOExceptionOccur@ 00000001800081f8     libfollowref003.obj
 0002:00001220       ??_C@_03OFAPEBGM@?$CFs?6@  0000000180008220     libfollowref003.obj
 0002:00001228       ??_C@_0DM@LPIGEGNJ@s?2test?2hotspot?2jtreg?2vmTestbase@ 0000000180008228     libfollowref003.obj
 0002:00001268       ??_C@_0CC@NFCNPEPK@Exception?5in?5JNI?5call?5?$CIcleared?$CJ@ 0000000180008268     libfollowref003.obj
 0002:00001290       ??_C@_0BJ@IBAKFIKF@jni?9?$DOExceptionDescribe?$CI?$CJ@ 0000000180008290     libfollowref003.obj
 0002:000012b0       ??_C@_0BG@GGKALKMH@jni?9?$DOExceptionClear?$CI?$CJ@ 00000001800082b0     libfollowref003.obj
 0002:000012c8       ??_C@_0CF@JMGFGJLJ@?$CD?5?5?5verified?5JNI?5assertion?5is?5F@ 00000001800082c8     libfollowref003.obj
 0002:000012f0       ??_C@_07KBAMPNJK@verbose@  00000001800082f0     libfollowref003.obj
 0002:000012f8       ??_C@_0DN@PKJBOLAP@nsk_jvmti_parseOptions?$CI?$CJ?3?5unexp@ 00000001800082f8     libfollowref003.obj
 0002:00001338       ??_C@_05IMBNNINJ@trace@    0000000180008338     libfollowref003.obj
 0002:00001340       ??_C@_0DD@BJKGNDMB@nsk_jvmti_parseOptions?$CI?$CJ?3?5no?5va@ 0000000180008340     libfollowref003.obj
 0002:00001374       ??_C@_04CGFJFPFD@none@     0000000180008374     libfollowref003.obj
 0002:0000137c       ??_C@_06BMELKFMA@before@   000000018000837c     libfollowref003.obj
 0002:00001384       ??_C@_05CMKPCFDK@after@    0000000180008384     libfollowref003.obj
 0002:0000138c       ??_C@_03NFKEKGGK@all@      000000018000838c     libfollowref003.obj
 0002:00001390       ??_C@_0DM@NDNJGJKE@nsk_jvmti_parseOptions?$CI?$CJ?3?5uexpe@ 0000000180008390     libfollowref003.obj
 0002:000013d0       ??_C@_08NBBJKJO@waittime@  00000001800083d0     libfollowref003.obj
 0002:000013e0       ??_C@_0DO@CMHGAOHC@nsk_jvmti_parseOptions?$CI?$CJ?3?5not?5i@ 00000001800083e0     libfollowref003.obj
 0002:00001420       ??_C@_0DL@LNMPBDLN@nsk_jvmti_parseOptions?$CI?$CJ?3?5negat@ 0000000180008420     libfollowref003.obj
 0002:00001460       ??_C@_0DA@GMFJNOJH@nsk_jvmti_parseOptions?$CI?$CJ?3?5unkno@ 0000000180008460     libfollowref003.obj
 0002:00001490       ??_C@_0CO@CCIAMEAN@nsk_jvmti_parseOptions?$CI?$CJ?3?5found@ 0000000180008490     libfollowref003.obj
 0002:000014c0       ??_C@_0CJ@OEGPCGDL@nsk_jvmti_parseOptions?$CI?$CJ?3?5out?5o@ 00000001800084c0     libfollowref003.obj
 0002:000014f0       ??_C@_0DI@NMBHPGGF@nsk_jvmti_parseOptions?$CI?$CJ?3?5too?5m@ 00000001800084f0     libfollowref003.obj
 0002:00001528       ??_C@_03POGCGECB@?5?0?$HO@ 0000000180008528     libfollowref003.obj
 0002:00001530       ??_C@_0DC@GKLNPJIJ@nsk_jvmti_findOptionValue?$CI?$CJ?3?5op@ 0000000180008530     libfollowref003.obj
 0002:00001568       ??_C@_0DF@OPPIHBPJ@nsk_jvmti_findOptionIntValue?$CI?$CJ?3@ 0000000180008568     libfollowref003.obj
 0002:000015a0       ??_C@_0DO@DBKDODPI@nsk_jvmti_findOptionIntValue?$CI?$CJ?3@ 00000001800085a0     libfollowref003.obj
 0002:000015e0       ??_C@_0EE@NGNPKOJC@nsk_jvmti_findOptionIntValue?$CI?$CJ?3@ 00000001800085e0     libfollowref003.obj
 0002:00001628       ??_C@_0CB@MLNJNCLJ@?5?5jvmti?5error?3?5code?$DN?$CFd?0?5name?$DN?$CFs@ 0000000180008628     libfollowref003.obj
 0002:00001650       ??_C@_0CD@OHBGDKMK@?$CD?5?5?5jvmti?5error?3?5code?$DN?$CFd?0?5name?$DN@ 0000000180008650     libfollowref003.obj
 0002:00001678       ??_C@_0CG@JNNCGPHB@?$CD?5?5?5error?5expected?3?5code?$DN?$CFd?0?5na@ 0000000180008678     libfollowref003.obj
 0002:000016a0       ??_C@_0EB@IMGKPCGE@?$CIstr_obj?5?$DN?5jni?9?$DONewStringUTF?$CIco@ 00000001800086a0     libfollowref003.obj
 0002:000016f0       ??_C@_0EA@HFOGGBCC@s?2test?2hotspot?2jtreg?2vmTestbase@ 00000001800086f0     libfollowref003.obj
 0002:00001730       ??_C@_05KKCIMGE@error@     0000000180008730     libfollowref003.obj
 0002:00001738       ??_C@_0CJ@JACLEAA@Test?5failed?5by?5setFailStatus?$CI?$CJ?4@ 0000000180008738     libfollowref003.obj
 0002:00001768       ??_C@_0BD@HGNAOMCP@agent_data_monitor@ 0000000180008768     libfollowref003.obj
 0002:00001780       ??_C@_0EB@OGCLGKLN@javaVM?9?$DOGetEnv?$CI?$CIvoid?5?$CK?$CK?$CJ?$CGjvmti_@ 0000000180008780     libfollowref003.obj
 0002:000017d0       ??_C@_0EA@PNBCDMOA@s?2test?2hotspot?2jtreg?2vmTestbase@ 00000001800087d0     libfollowref003.obj
 0002:00001810       ??_C@_0CI@DDPIFBGM@init_agent_data?$CIjvmti_env?0?5?$CGage@ 0000000180008810     libfollowref003.obj
 0002:00001838       ??_C@_0DI@ILAHDLMP@?$CI?$CKagentThreadProc?$CJ?$CIjvmti_env?0?5a@ 0000000180008838     libfollowref003.obj
 0002:00001870       ??_C@_0BD@KDBALNLB@JVMTI?5agent?5thread@ 0000000180008870     libfollowref003.obj
 0002:00001888       ??_C@_0BB@NOKBFPFO@java?1lang?1Thread@ 0000000180008888     libfollowref003.obj
 0002:0000189c       ??_C@_06FALKBLGB@?$DMinit?$DO@ 000000018000889c     libfollowref003.obj
 0002:000018a8       ??_C@_0BG@IKDDPPGD@?$CILjava?1lang?1String?$DL?$CJV@ 00000001800088a8     libfollowref003.obj
 0002:000018c0       ??_C@_0EB@IFJBFEKC@?$CIthreadClass?5?$DN?5jni_env?9?$DOFindCla@ 00000001800088c0     libfollowref003.obj
 0002:00001910       ??_C@_0GF@FGFIBKKL@?$CIthreadCtor?5?$DN?5jni_env?9?$DOGetMetho@ 0000000180008910     libfollowref003.obj
 0002:00001978       ??_C@_0DN@NCPDJLOG@?$CIthreadName?5?$DN?5jni_env?9?$DONewStrin@ 0000000180008978     libfollowref003.obj
 0002:000019c0       ??_C@_0FE@PFKODBGC@?$CIthreadObject?5?$DN?5jni_env?9?$DONewObj@ 00000001800089c0     libfollowref003.obj
 0002:00001a20       ??_C@_0ED@HOBAHHJI@?$CIthreadGlobalRef?5?$DN?5jni_env?9?$DONew@ 0000000180008a20     libfollowref003.obj
 0002:00001a70       ??_C@_0FN@HNJJAHFC@jvmti_env?9?$DORunAgentThread?$CIagent@ 0000000180008a70     libfollowref003.obj
 0002:00001ad0       ??_C@_0EA@MOJDNKDF@Debuggee?5status?5sync?5aborted?5be@ 0000000180008ad0     libfollowref003.obj
 0002:00001b10       ??_C@_0CO@PGPGMHBJ@No?5status?5sync?5occured?5for?5time@ 0000000180008b10     libfollowref003.obj
 0002:00001b40       ??_C@_0CL@DOEBDPKJ@Debuggee?5was?5not?5suspended?5on?5s@ 0000000180008b40     libfollowref003.obj
 0002:00001b70       ??_C@_0EA@EEOEJAEN@status?5?$DN?5syncDebuggeeStatus?$CIjni@ 0000000180008b70     libfollowref003.obj
 0002:00001bb0       ??_C@_0BL@JBCFNBMB@nsk_jvmti_resetAgentData?$CI?$CJ@ 0000000180008bb0     libfollowref003.obj
 0002:00001bd0       ??_C@_0EL@LPBEELIP@s?2test?2hotspot?2jtreg?2vmTestbase@ 0000000180008bd0     libfollowref003.obj
 0002:00001c20       ??_C@_0CK@JDAMFDMJ@jvmti?9?$DOSetTag?$CIo?0?5tag?$CJ?5?$DN?$DN?5JVMTI_@ 0000000180008c20     libfollowref003.obj
 0002:00001c50       ??_C@_0CC@DAMNHKNI@Can?8t?5set?5tag?5?$CFli?5for?5object?5?$CFl@ 0000000180008c50     libfollowref003.obj
 0002:00001c78       ??_C@_0DL@HAJPNKEF@jvmti?9?$DOGetObjectHashCode?$CIo?0?5?$CGha@ 0000000180008c78     libfollowref003.obj
 0002:00001cb8       ??_C@_0BL@JFPIEOBF@Can?8t?5get?5hash?5object?5?$CFlx?6@ 0000000180008cb8     libfollowref003.obj
 0002:00001cd8       ??_C@_0BG@DICPHBKN@setTag?3?5?$CF08x?5?$DM?9?5?$CF?53li@ 0000000180008cd8     libfollowref003.obj
 0002:00001cf0       ??_C@_0DH@FCEEBDMJ@?$CIs?5?$DN?5jni?9?$DOGetStringUTFChars?$CIsIn@ 0000000180008cf0     libfollowref003.obj
 0002:00001d28       ??_C@_0BJ@OKKGHDCN@Can?8t?5get?5string?5at?5?$CF?$CDp?6@ 0000000180008d28     libfollowref003.obj
 0002:00001d48       ??_C@_0BP@EKFLGGFJ@Can?8t?5get?5string?5at?5?$CF?$CDp?3?5null?6@ 0000000180008d48     libfollowref003.obj
 0002:00001d68       ??_C@_06ICODBHCL@?5?1?1?5?$CFs@ 0000000180008d68     libfollowref003.obj
 0002:00001d70       ??_C@_0DB@KGFPLEGO@?$CIr?5?$DN?5jvmti?9?$DOGetTag?$CIo?0?5?$CGtag?$CJ?$CJ?5?$DN?$DN@ 0000000180008d70     libfollowref003.obj
 0002:00001da8       ??_C@_0CO@PDAGBCGJ@Can?8t?5GetTag?5for?5object?5?$CFlx?4?5Re@ 0000000180008da8     libfollowref003.obj
 0002:00001dd8       ??_C@_0CH@HPEODOHC@TEST_BUG?3?5Max?4?5number?5of?5refs?5r@ 0000000180008dd8     libfollowref003.obj
 0002:00001e00       ??_C@_0DI@PHFCABIM@?$CIr?5?$DN?5jvmti?9?$DOGetTag?$CIfrom?0?5?$CGtagFr@ 0000000180008e00     libfollowref003.obj
 0002:00001e38       ??_C@_0DI@MDEGFNKD@TEST_BUG?3?5Can?8t?5GetTag?5for?5obje@ 0000000180008e38     libfollowref003.obj
 0002:00001e70       ??_C@_0DE@MLELJAHM@?$CIr?5?$DN?5jvmti?9?$DOGetTag?$CIto?0?5?$CGtagTo?$CJ?$CJ@ 0000000180008e70     libfollowref003.obj
 0002:00001eb0       ??_C@_0EA@OLCLFBLL@?$CIobj?5?$DN?5jni?9?$DOGetObjectField?$CIfirs@ 0000000180008eb0     libfollowref003.obj
 0002:00001ef0       ??_C@_0FO@BJBNCGGE@s?2test?2hotspot?2jtreg?2vmTestbase@ 0000000180008ef0     libfollowref003.obj
 0002:00001f50       ??_C@_0BL@HDOCIPLI@jvmti?9?$DOSetTag?$CIobj?0?5objTag?$CJ@ 0000000180008f50     libfollowref003.obj
 0002:00001f70       ??_C@_0BP@KLIOMM@?5?5?5?5?5?5?5?5tag?$DN?$CF?95ld?5object?$DN0x?$CFp?6@ 0000000180008f70     libfollowref003.obj
 0002:00001f90       ??_C@_0BJ@NBEMCAEP@jni?9?$DODeleteLocalRef?$CIobj?$CJ@ 0000000180008f90     libfollowref003.obj
 0002:00001fb0       ??_C@_0CO@OFDFJEOH@Allocate?5memory?5for?5objects?5lis@ 0000000180008fb0     libfollowref003.obj
 0002:00001fe0       ??_C@_0FH@KENAHJKN@jvmti?9?$DOAllocate?$CI?$CI?$CKobjectsCount?5@ 0000000180008fe0     libfollowref003.obj
 0002:00002038       ??_C@_0BN@GHDOCCDB@?5?5?4?4?4?5allocated?5array?3?50x?$CFp?6@ 0000000180009038     libfollowref003.obj
 0002:00002058       ??_C@_0CN@FGPKEMCO@nsk?1jvmti?1unit?1FollowReferences@ 0000000180009058     libfollowref003.obj
 0002:00002088       ??_C@_0BI@ENEOJHP@Find?5debugee?5class?3?5?$CFs?6@ 0000000180009088     libfollowref003.obj
 0002:000020a0       ??_C@_0DP@MFMMLPOM@?$CIdebugeeClass?5?$DN?5jni?9?$DOFindClass?$CI@ 00000001800090a0     libfollowref003.obj
 0002:000020e0       ??_C@_0BJ@DFGCANJI@?5?5?4?4?4?5found?5class?3?50x?$CFp?6@ 00000001800090e0     libfollowref003.obj
 0002:00002100       ??_C@_0DM@EJDKHJGM@nsk?1jvmti?1unit?1FollowReferences@ 0000000180009100     libfollowref003.obj
 0002:00002140       ??_C@_0BM@GFHMIOD@Find?5root?5object?5class?3?5?$CFs?6@ 0000000180009140     libfollowref003.obj
 0002:00002160       ??_C@_0EG@LBKAPJFG@?$CIrootObjectClass?5?$DN?5jni?9?$DOFindCla@ 0000000180009160     libfollowref003.obj
 0002:000021a8       ??_C@_0CN@GCKFBJII@jvmti?9?$DOSetTag?$CIrootObjectClass?0?5@ 00000001800091a8     libfollowref003.obj
 0002:000021d8       ??_C@_0CC@HGDALAOA@?5?5?5?5?5?5?5?5tag?$DN?$CF?95ld?5rootClass?$DN0x?$CF@ 00000001800091d8     libfollowref003.obj
 0002:00002200       ??_C@_0DI@INPBEPAM@nsk?1jvmti?1unit?1FollowReferences@ 0000000180009200     libfollowref003.obj
 0002:00002238       ??_C@_0BN@JPFPOKGN@Find?5chain?5object?5class?3?5?$CFs?6@ 0000000180009238     libfollowref003.obj
 0002:00002260       ??_C@_0EI@PFABFCAO@?$CIchainObjectClass?5?$DN?5jni?9?$DOFindCl@ 0000000180009260     libfollowref003.obj
 0002:000022a8       ??_C@_0CP@DMFCGFKG@jvmti?9?$DOSetTag?$CIchainObjectClass?0@ 00000001800092a8     libfollowref003.obj
 0002:000022d8       ??_C@_0CD@KGGDJHOJ@?5?5?5?5?5?5?5?5tag?$DN?$CF?95ld?5chainClass?$DN0x@ 00000001800092d8     libfollowref003.obj
 0002:000022fc       ??_C@_06IEOJBDIK@object@   00000001800092fc     libfollowref003.obj
 0002:00002308       ??_C@_0CI@IPDCJCKO@Find?5static?5field?5in?5debugee?5cl@ 0000000180009308     libfollowref003.obj
 0002:00002330       ??_C@_0GJ@EJPDBEIJ@?$CIobjectField?5?$DN?5jni?9?$DOGetStaticFi@ 0000000180009330     libfollowref003.obj
 0002:000023a0       ??_C@_0DO@DICFCANO@Lnsk?1jvmti?1unit?1FollowReference@ 00000001800093a0     libfollowref003.obj
 0002:000023e0       ??_C@_0BJ@MIIADDIH@?5?5?4?4?4?5got?5fieldID?3?50x?$CFp?6@ 00000001800093e0     libfollowref003.obj
 0002:00002400       ??_C@_0P@OFCAMOEL@reachableChain@ 0000000180009400     libfollowref003.obj
 0002:00002410       ??_C@_0CO@GJFDOONJ@Find?5instance?5field?5in?5root?5obj@ 0000000180009410     libfollowref003.obj
 0002:00002440       ??_C@_0HI@JPPGJND@?$CIreachableChainField?5?$DN?5jni?9?$DOGet@ 0000000180009440     libfollowref003.obj
 0002:000024b8       ??_C@_0DK@ODGKBEJD@Lnsk?1jvmti?1unit?1FollowReference@ 00000001800094b8     libfollowref003.obj
 0002:000024f8       ??_C@_0BB@HCMFGFMC@unreachableChain@ 00000001800094f8     libfollowref003.obj
 0002:00002510       ??_C@_0HM@FNOMFGGD@?$CIunreachableChainField?5?$DN?5jni?9?$DOG@ 0000000180009510     libfollowref003.obj
 0002:0000258c       ??_C@_04DIFLAKIP@tail@     000000018000958c     libfollowref003.obj
 0002:00002598       ??_C@_0CP@FJDMDHPJ@Find?5instance?5field?5in?5chain?5ob@ 0000000180009598     libfollowref003.obj
 0002:000025d0       ??_C@_0GE@BFDKKHME@?$CItailField?5?$DN?5jni?9?$DOGetFieldID?$CIch@ 00000001800095d0     libfollowref003.obj
 0002:00002638       ??_C@_0CH@IEEMMCJA@Get?5root?5object?5from?5static?5fie@ 0000000180009638     libfollowref003.obj
 0002:00002660       ??_C@_0FA@EKCCJLK@?$CI?$CKrootObject?5?$DN?5jni?9?$DOGetStaticOb@ 0000000180009660     libfollowref003.obj
 0002:000026b0       ??_C@_0BI@FNLCMIKO@?5?5?4?4?4?5got?5object?3?50x?$CFp?6@ 00000001800096b0     libfollowref003.obj
 0002:000026c8       ??_C@_0DK@BGLMLPLF@?$CI?$CKrootObject?5?$DN?5jni?9?$DONewGlobalRe@ 00000001800096c8     libfollowref003.obj
 0002:00002708       ??_C@_0BI@DDGFIBLM@?5?5?4?4?4?5global?5ref?3?50x?$CFp?6@ 0000000180009708     libfollowref003.obj
 0002:00002720       ??_C@_0BP@MAGAMBHE@Obtain?5and?5tag?5chain?5objects?3?6@ 0000000180009720     libfollowref003.obj
 0002:00002740       ??_C@_0BI@DBPLAMDB@?5?5?5?5root?5tested?5object?6@ 0000000180009740     libfollowref003.obj
 0002:00002758       ??_C@_0CK@FKPEDLDC@jvmti?9?$DOSetTag?$CI?$CKrootObject?0?5root@ 0000000180009758     libfollowref003.obj
 0002:00002788       ??_C@_0CJ@ELCOJLPK@?5?5?5?5reachable?5objects?5chain?3?5?$CFd@ 0000000180009788     libfollowref003.obj
 0002:000027b8       ??_C@_0CL@LBFMJNLN@?5?5?5?5unreachable?5objects?5chain?3?5@ 00000001800097b8     libfollowref003.obj
 0002:000027e8       ??_C@_0CJ@OGMDHCIM@Following?5tagged?5objects?5were?5i@ 00000001800097e8     libfollowref003.obj
 0002:00002818       ??_C@_0BF@HEOKDGAN@Root?5tested?5object?3?6@ 0000000180009818     libfollowref003.obj
 0002:00002830       ??_C@_0FP@HPNCGAGF@?5?5?5tag?3?5?5?5?5?5?5?5?5?5?5?5?5?5?5?5?5?5?$CFld?6?5?5?5@ 0000000180009830     libfollowref003.obj
 0002:00002890       ??_C@_0DD@EPIDJGDN@Root?5tested?5object?5unexpectedly@ 0000000180009890     libfollowref003.obj
 0002:000028c8       ??_C@_0BF@IBKKIPPL@?6Reachable?5objects?3?6@ 00000001800098c8     libfollowref003.obj
 0002:000028e0       ??_C@_0HD@CEGHGPK@Reachable?5object?3?6?5?5?5tag?3?5?5?5?5?5?5@ 00000001800098e0     libfollowref003.obj
 0002:00002958       ??_C@_0CD@KFMGLHOH@Reachable?5object?5was?5not?5iterat@ 0000000180009958     libfollowref003.obj
 0002:00002980       ??_C@_0DK@MMBLMPDO@Reachable?5object?5was?5iterated?5u@ 0000000180009980     libfollowref003.obj
 0002:000029c0       ??_C@_0BH@BMDNFMCE@?6Unreachable?5objects?3?6@ 00000001800099c0     libfollowref003.obj
 0002:000029e0       ??_C@_0HD@MFBDFDHC@Unreachable?5object?3?6?5?5?5tag?3?5?5?5?5@ 00000001800099e0     libfollowref003.obj
 0002:00002a58       ??_C@_0CB@KMMKJGIO@Unreachable?5object?5was?5iterated@ 0000000180009a58     libfollowref003.obj
 0002:00002a80       ??_C@_0DG@ONNGGIGA@Release?5object?5reference?5to?5roo@ 0000000180009a80     libfollowref003.obj
 0002:00002ab8       ??_C@_0CB@MNNHEDND@jni?9?$DODeleteGlobalRef?$CIrootObject@ 0000000180009ab8     libfollowref003.obj
 0002:00002ae0       ??_C@_0BP@JPEMGJLC@Deallocate?5objects?5list?3?50x?$CFp?6@ 0000000180009ae0     libfollowref003.obj
 0002:00002b00       ??_C@_0DC@DFJJAFOM@jvmti?9?$DODeallocate?$CI?$CIunsigned?5cha@ 0000000180009b00     libfollowref003.obj
 0002:00002b38       ??_C@_0BL@INMGEMCA@Unexpected?5thread?5ID?3?5?$CFld?6@ 0000000180009b38     libfollowref003.obj
 0002:00002b60       ??_C@_0GD@NKPAGPKM@Thread?5tag?5doesn?8t?5match?5the?5fi@ 0000000180009b60     libfollowref003.obj
 0002:00002bc8       ??_C@_0BM@FCIIEHHC@Incorrect?5frame?5depth?3?5?$CFld?6@ 0000000180009bc8     libfollowref003.obj
 0002:00002be8       ??_C@_0BL@BOHHMIAO@methodID?5must?5not?5be?5null?6@ 0000000180009be8     libfollowref003.obj
 0002:00002c08       ??_C@_0CP@ONCBHECC@Internal?3?5Insufficient?5frames?5t@ 0000000180009c08     libfollowref003.obj
 0002:00002c38       ??_C@_0CC@NAKLNLGB@Incorrect?5stack?5local?5slot?$CD?3?5?$CFl@ 0000000180009c38     libfollowref003.obj
 0002:00002c60       ??_C@_0BJ@PPEHNMPK@Location?5must?5not?5be?5?91?6@ 0000000180009c60     libfollowref003.obj
 0002:00002c80       ??_C@_0DO@OLEAJABP@Second?5report?5of?5the?5local?3?5loc@ 0000000180009c80     libfollowref003.obj
 0002:00002cc0       ??_C@_0CF@CPPLCGD@?7?5thr_id?$DN?$CFI64d?0?5depth?$DN?$CFd?0?5meth?$DN@ 0000000180009cc0     libfollowref003.obj
 0002:00002ce8       ??_C@_0DA@CDEGLNKE@Tag?5mismatch?3?5?5?5?5?5?5expected?5?$CF?$CDl@ 0000000180009ce8     libfollowref003.obj
 0002:00002d18       ??_C@_0CO@HONPGMIO@Location?5mismatch?3?5expected?5?$CFld@ 0000000180009d18     libfollowref003.obj
 0002:00002d48       ??_C@_0CO@NDOMFGAK@Internal?3?5Insufficient?5locals?5t@ 0000000180009d48     libfollowref003.obj
 0002:00002d78       ??_C@_0DL@GILACKOJ@?5?5?5?5?5heapReferenceCallback?3?5ref@ 0000000180009d78     libfollowref003.obj
 0002:00002dc0       ??_C@_0KC@FOJPFHLO@?5?5?5?5?5heapReferenceCallback?3?5ref@ 0000000180009dc0     libfollowref003.obj
 0002:00002e68       ??_C@_0DP@PIPPEBCM@null?5tag_ptr?5is?5passed?5to?5heapR@ 0000000180009e68     libfollowref003.obj
 0002:00002ea8       ??_C@_0DO@FEAPJGEB@Unreachable?5tagged?5object?5is?5pa@ 0000000180009ea8     libfollowref003.obj
 0002:00002ee8       ??_C@_0DK@CGCKBBLN@Unknown?5tagged?5object?5is?5passed@ 0000000180009ee8     libfollowref003.obj
 0002:00002f30       ??_C@_0GK@JFIMNGPJ@Unexpected?5user_data?5is?5passed?5@ 0000000180009f30     libfollowref003.obj
 0002:00002fa0       ??_C@_0DJ@LKLDKLNP@Unknown?5tagged?5class?5is?5passed?5@ 0000000180009fa0     libfollowref003.obj
 0002:00002fe0       ??_C@_0GA@GBOLFLEP@Wrong?5tag?5in?5heapReferenceCallb@ 0000000180009fe0     libfollowref003.obj
 0002:00003040       ??_C@_0CK@FJOIAFDI@This?5reference?5kind?5was?5not?5exp@ 000000018000a040     libfollowref003.obj
 0002:00003070       ??_C@_0DN@KHHLPFNM@Wrong?5length?5of?5the?5local?5array@ 000000018000a070     libfollowref003.obj
 0002:000030b0       ??_C@_0CA@GHCCMD@Length?5of?5array?5must?5not?5be?5?91?6@ 000000018000a0b0     libfollowref003.obj
 0002:000030d0       ??_C@_0CL@NCLELIBB@This?5reference?5kind?5was?5not?5exp@ 000000018000a0d0     libfollowref003.obj
 0002:00003100       ??_C@_0EG@EIHEEGH@?5primitiveFieldCallback?3?5ref?$DN?$CFs@ 000000018000a100     libfollowref003.obj
 0002:00003150       ??_C@_0EL@PGAOEPDL@?5arrayPrimitiveValueCallback?3?5c@ 000000018000a150     libfollowref003.obj
 0002:000031a0       ??_C@_0EC@DNGCCNKG@stringPrimitiveValueCallback?3?5c@ 000000018000a1a0     libfollowref003.obj
 0002:000031e4       ??_C@_04GHJNJNPO@main@     000000018000a1e4     libfollowref003.obj
 0002:000031f0       ??_C@_0CB@KHPCBPAO@Wait?5for?5tested?5objects?5created@ 000000018000a1f0     libfollowref003.obj
 0002:00003218       ??_C@_0BP@LAIJOMPC@nsk_jvmti_waitForSync?$CItimeout?$CJ@ 000000018000a218     libfollowref003.obj
 0002:00003238       ??_C@_0DG@CILGJCLA@?$DO?$DO?$DO?5Obtain?5and?5tag?5tested?5objec@ 000000018000a238     libfollowref003.obj
 0002:00003270       ??_C@_0FH@DCIANFHH@getTestedObjects?$CIjvmti?0?5jni?0?5ch@ 000000018000a270     libfollowref003.obj
 0002:000032c8       ??_C@_0DH@PBGGKADM@?$DO?$DO?$DO?5Let?5debugee?5to?5clean?5links?5@ 000000018000a2c8     libfollowref003.obj
 0002:00003300       ??_C@_0BH@LECMGIIA@nsk_jvmti_resumeSync?$CI?$CJ@ 000000018000a300     libfollowref003.obj
 0002:00003318       ??_C@_0CO@JGMAHOPB@setTagForTargetThread?$CIjvmti?0?5TA@ 000000018000a318     libfollowref003.obj
 0002:00003348       ??_C@_0DI@HJIOHFDI@?6?6?$DO?$DO?$DO?5Start?51?9st?5iteration?5star@ 000000018000a348     libfollowref003.obj
 0002:00003380       ??_C@_0HF@CGLOJNDD@jvmti?9?$DOFollowReferences?$CI?$CIjint?$CJ?5@ 000000018000a380     libfollowref003.obj
 0002:000033f8       ??_C@_0CO@NJMAAGEM@?$DO?$DO?$DO?5Check?5if?5reachable?5objects?5@ 000000018000a3f8     libfollowref003.obj
 0002:00003428       ??_C@_0DI@POGMFMK@?6?6?$DO?$DO?$DO?5Start?52?9nd?5iteration?5star@ 000000018000a428     libfollowref003.obj
 0002:00003460       ??_C@_0HI@DKHILCG@jvmti?9?$DOFollowReferences?$CIheap_fi@ 000000018000a460     libfollowref003.obj
 0002:000034e0       ??_C@_0EJ@DLJDCAFG@?$DO?$DO?$DO?5Check?5that?5both?5reachable?5a@ 000000018000a4e0     libfollowref003.obj
 0002:00003530       ??_C@_0BF@MNKEFEOE@?$DO?$DO?$DO?5Clean?5used?5data?6@ 000000018000a530     libfollowref003.obj
 0002:00003550       ??_C@_0EK@LKBLLAJH@releaseTestedObjects?$CIjvmti?0?5jni@ 000000018000a550     libfollowref003.obj
 0002:000035a0       ??_C@_0BH@HPEOJMHL@Let?5debugee?5to?5finish?6@ 000000018000a5a0     libfollowref003.obj
 0002:000035b8       ??_C@_0CA@MNKGCBCG@nsk_jvmti_parseOptions?$CIoptions?$CJ@ 000000018000a5b8     libfollowref003.obj
 0002:000035d8       ??_C@_04NIDJFNBE@info@     000000018000a5d8     libfollowref003.obj
 0002:000035e0       ??_C@_06DFFOHAMN@objref@   000000018000a5e0     libfollowref003.obj
 0002:000035e8       ??_C@_08JAMFKCP@stackref@  000000018000a5e8     libfollowref003.obj
 0002:000035f8       ??_C@_08KICKEILH@heaproot@ 000000018000a5f8     libfollowref003.obj
 0002:00003608       ??_C@_07MNCDLPNM@heapobj@  000000018000a608     libfollowref003.obj
 0002:00003610       ??_C@_0BP@PNAOMHNJ@Unknown?5option?5value?3?5info?$DN?$CFs?6@ 000000018000a610     libfollowref003.obj
 0002:00003630       ??_C@_07JPLKJBI@objects@   000000018000a630     libfollowref003.obj
 0002:00003638       ??_C@_0BA@LIAABLEG@chainLength?5?$DO?50@ 000000018000a638     libfollowref003.obj
 0002:00003648       ??_C@_0DN@MIAMNFPH@?$CIjvmti?5?$DN?5nsk_jvmti_createJVMTIE@ 000000018000a648     libfollowref003.obj
 0002:00003688       ??_C@_0BO@DBKDIPGD@jvmti?9?$DOAddCapabilities?$CI?$CGcaps?$CJ@ 000000018000a688     libfollowref003.obj
 0002:000036a8       ??_C@_0CL@PIACJIPK@nsk_jvmti_setAgentProc?$CIagentPro@ 000000018000a6a8     libfollowref003.obj
 0002:000036f0       ??_C@_1EC@JIJBPKFM@?$AAa?$AAp?$AAi?$AA?9?$AAm?$AAs?$AA?9?$AAw?$AAi?$AAn?$AA?9?$AAc?$AAo?$AAr?$AAe@ 000000018000a6f0     MSVCRT:thread_safe_statics.obj
 0002:00003738       ??_C@_1BK@MGMFAEKH@?$AAk?$AAe?$AAr?$AAn?$AAe?$AAl?$AA3?$AA2?$AA?4?$AAd?$AAl?$AAl@ 000000018000a738     MSVCRT:thread_safe_statics.obj
 0002:00003758       ??_C@_0BJ@JEBJOJFJ@SleepConditionVariableCS@ 000000018000a758     MSVCRT:thread_safe_statics.obj
 0002:00003778       ??_C@_0BJ@PGPPEPCC@WakeAllConditionVariable@ 000000018000a778     MSVCRT:thread_safe_statics.obj
 0002:00003798       _pDefaultRawDllMain        000000018000a798     MSVCRT:dll_dllmain.obj
 0002:00003798       _pRawDllMain               000000018000a798     MSVCRT:dll_dllmain.obj
 0002:000037a0       __xmm@ffffffffffffffffffffffffffffffff 000000018000a7a0     MSVCRT:utility.obj
 0002:000037b0       _load_config_used          000000018000a7b0     MSVCRT:loadcfg.obj
 0002:00003980       _tls_used                  000000018000a980     MSVCRT:tlssup.obj
 0002:000039a8       __volatile_metadata        000000018000a9a8     <linker-defined>
 0002:00003d80       __rtc_iaa                  000000018000ad80     MSVCRT:initsect.obj
 0002:00003d88       __rtc_izz                  000000018000ad88     MSVCRT:initsect.obj
 0002:00003d90       __rtc_taa                  000000018000ad90     MSVCRT:initsect.obj
 0002:00003d98       __rtc_tzz                  000000018000ad98     MSVCRT:initsect.obj
 0002:00003da0       _tls_start                 000000018000ada0     MSVCRT:tlssup.obj
 0002:00003da4       _Init_thread_epoch         000000018000ada4     MSVCRT:thread_safe_statics.obj
 0002:00003da8       _tls_end                   000000018000ada8     MSVCRT:tlssup.obj
 0002:00004514       __IMPORT_DESCRIPTOR_KERNEL32 000000018000b514     kernel32:KERNEL32.dll
 0002:00004528       __IMPORT_DESCRIPTOR_VCRUNTIME140 000000018000b528     vcruntime:VCRUNTIME140.dll
 0002:0000453c       __IMPORT_DESCRIPTOR_api-ms-win-crt-heap-l1-1-0 000000018000b53c     ucrt:api-ms-win-crt-heap-l1-1-0.dll
 0002:00004550       __IMPORT_DESCRIPTOR_api-ms-win-crt-runtime-l1-1-0 000000018000b550     ucrt:api-ms-win-crt-runtime-l1-1-0.dll
 0002:00004564       __IMPORT_DESCRIPTOR_api-ms-win-crt-convert-l1-1-0 000000018000b564     ucrt:api-ms-win-crt-convert-l1-1-0.dll
 0002:00004578       __IMPORT_DESCRIPTOR_api-ms-win-crt-stdio-l1-1-0 000000018000b578     ucrt:api-ms-win-crt-stdio-l1-1-0.dll
 0002:0000458c       __IMPORT_DESCRIPTOR_api-ms-win-crt-string-l1-1-0 000000018000b58c     ucrt:api-ms-win-crt-string-l1-1-0.dll
 0002:000045a0       __NULL_IMPORT_DESCRIPTOR   000000018000b5a0     kernel32:KERNEL32.dll
 0003:00000148       _Init_global_epoch         000000018000c148     MSVCRT:thread_safe_statics.obj
 0003:00000150       __security_cookie          000000018000c150     MSVCRT:gs_cookie.obj
 0003:00000158       __security_cookie_complement 000000018000c158     MSVCRT:gs_cookie.obj
 0003:00000160       __scrt_native_dllmain_reason 000000018000c160     MSVCRT:utility.obj
 0003:00000168       __isa_available            000000018000c168     MSVCRT:cpu_disp.obj
 0003:0000016c       __isa_enabled              000000018000c16c     MSVCRT:cpu_disp.obj
 0003:00000170       __memset_fast_string_threshold 000000018000c170     MSVCRT:cpu_disp.obj
 0003:00000178       __memset_nt_threshold      000000018000c178     MSVCRT:cpu_disp.obj
 0003:00000180       __scrt_ucrt_dll_is_in_use  000000018000c180     MSVCRT:ucrt_stubs.obj
 0003:00000190       g_wrongHeapCallbacks       000000018000c190     libfollowref003.obj
 0003:00000210       g_szTagInfo                000000018000c210     libfollowref003.obj
 0003:00002150       g_tagFlags                 000000018000e150     libfollowref003.obj
 0003:00002538       g_refsToVerifyCnt          000000018000e538     libfollowref003.obj
 0003:0000253c       g_fakeUserData             000000018000e53c     libfollowref003.obj
 0003:00002540       g_tagVisitCount            000000018000e540     libfollowref003.obj
 0003:000034e0       g_refsToVerify             000000018000f4e0     libfollowref003.obj
 0003:0001abe0       g_userDataError            0000000180026be0     libfollowref003.obj
 0003:000212a0       ?_OptionsStorage@?1??__local_stdio_printf_options@@9@4_KA 000000018002d2a0     libfollowref003.obj
 0003:00021868       _tls_index                 000000018002d868     MSVCRT:tlssup.obj
 0003:00021870       __scrt_current_native_startup_state 000000018002d870     MSVCRT:utility.obj
 0003:00021878       __scrt_native_startup_lock 000000018002d878     MSVCRT:utility.obj
 0003:000218b8       __scrt_debugger_hook_flag  000000018002d8b8     MSVCRT:utility_desktop.obj
 0003:000218c0       ?__type_info_root_node@@3U__type_info_node@@A 000000018002d8c0     MSVCRT:tncleanup.obj
 0003:000218d0       ?_OptionsStorage@?1??__local_stdio_scanf_options@@9@4_KA 000000018002d8d0     MSVCRT:default_local_stdio_options.obj
 0003:000218d8       __favor                    000000018002d8d8     MSVCRT:cpu_disp.obj
 0003:000218e0       __dyn_tls_init_callback    000000018002d8e0     <common>

 entry point at        0001:00004b20

 Static symbols

 0000:fffd0000       .debug$S                   0000000180000000     followref003.exp
 0000:fffd0000       .debug$S                   0000000180000000     vcruntime:VCRUNTIME140.dll
 0000:fffd0000       .debug$S                   0000000180000000     vcruntime:VCRUNTIME140.dll
 0000:fffd0000       .debug$S                   0000000180000000     vcruntime:VCRUNTIME140.dll
 0000:fffd0000       .debug$S                   0000000180000000     vcruntime:VCRUNTIME140.dll
 0000:fffd0000       .debug$S                   0000000180000000     vcruntime:VCRUNTIME140.dll
 0000:fffd0000       .debug$S                   0000000180000000     vcruntime:VCRUNTIME140.dll
 0000:fffd0000       .debug$S                   0000000180000000     vcruntime:VCRUNTIME140.dll
 0000:fffd0000       .debug$S                   0000000180000000     ucrt:api-ms-win-crt-convert-l1-1-0.dll
 0000:fffd0000       .debug$S                   0000000180000000     ucrt:api-ms-win-crt-heap-l1-1-0.dll
 0000:fffd0000       .debug$S                   0000000180000000     ucrt:api-ms-win-crt-heap-l1-1-0.dll
 0000:fffd0000       .debug$S                   0000000180000000     ucrt:api-ms-win-crt-heap-l1-1-0.dll
 0000:fffd0000       .debug$S                   0000000180000000     ucrt:api-ms-win-crt-heap-l1-1-0.dll
 0000:fffd0000       .debug$S                   0000000180000000     ucrt:api-ms-win-crt-runtime-l1-1-0.dll
 0000:fffd0000       .debug$S                   0000000180000000     ucrt:api-ms-win-crt-runtime-l1-1-0.dll
 0000:fffd0000       .debug$S                   0000000180000000     ucrt:api-ms-win-crt-runtime-l1-1-0.dll
 0000:fffd0000       .debug$S                   0000000180000000     ucrt:api-ms-win-crt-runtime-l1-1-0.dll
 0000:fffd0000       .debug$S                   0000000180000000     ucrt:api-ms-win-crt-runtime-l1-1-0.dll
 0000:fffd0000       .debug$S                   0000000180000000     ucrt:api-ms-win-crt-runtime-l1-1-0.dll
 0000:fffd0000       .debug$S                   0000000180000000     ucrt:api-ms-win-crt-runtime-l1-1-0.dll
 0000:fffd0000       .debug$S                   0000000180000000     ucrt:api-ms-win-crt-runtime-l1-1-0.dll
 0000:fffd0000       .debug$S                   0000000180000000     ucrt:api-ms-win-crt-runtime-l1-1-0.dll
 0000:fffd0000       .debug$S                   0000000180000000     ucrt:api-ms-win-crt-runtime-l1-1-0.dll
 0000:fffd0000       .debug$S                   0000000180000000     ucrt:api-ms-win-crt-runtime-l1-1-0.dll
 0000:fffd0000       .debug$S                   0000000180000000     ucrt:api-ms-win-crt-runtime-l1-1-0.dll
 0000:fffd0000       .debug$S                   0000000180000000     ucrt:api-ms-win-crt-runtime-l1-1-0.dll
 0000:fffd0000       .debug$S                   0000000180000000     ucrt:api-ms-win-crt-runtime-l1-1-0.dll
 0000:fffd0000       .debug$S                   0000000180000000     ucrt:api-ms-win-crt-runtime-l1-1-0.dll
 0000:fffd0000       .debug$S                   0000000180000000     ucrt:api-ms-win-crt-runtime-l1-1-0.dll
 0000:fffd0000       .debug$S                   0000000180000000     ucrt:api-ms-win-crt-stdio-l1-1-0.dll
 0000:fffd0000       .debug$S                   0000000180000000     ucrt:api-ms-win-crt-stdio-l1-1-0.dll
 0000:fffd0000       .debug$S                   0000000180000000     ucrt:api-ms-win-crt-stdio-l1-1-0.dll
 0000:fffd0000       .debug$S                   0000000180000000     ucrt:api-ms-win-crt-stdio-l1-1-0.dll
 0000:fffd0000       .debug$S                   0000000180000000     ucrt:api-ms-win-crt-stdio-l1-1-0.dll
 0000:fffd0000       .debug$S                   0000000180000000     ucrt:api-ms-win-crt-stdio-l1-1-0.dll
 0000:fffd0000       .debug$S                   0000000180000000     ucrt:api-ms-win-crt-stdio-l1-1-0.dll
 0000:fffd0000       .debug$S                   0000000180000000     ucrt:api-ms-win-crt-stdio-l1-1-0.dll
 0000:fffd0000       .debug$S                   0000000180000000     ucrt:api-ms-win-crt-stdio-l1-1-0.dll
 0000:fffd0000       .debug$S                   0000000180000000     ucrt:api-ms-win-crt-stdio-l1-1-0.dll
 0000:fffd0000       .debug$S                   0000000180000000     ucrt:api-ms-win-crt-string-l1-1-0.dll
 0000:fffd0000       .debug$S                   0000000180000000     ucrt:api-ms-win-crt-string-l1-1-0.dll
 0000:fffd0000       .debug$S                   0000000180000000     ucrt:api-ms-win-crt-string-l1-1-0.dll
 0000:fffd0000       .debug$S                   0000000180000000     ucrt:api-ms-win-crt-string-l1-1-0.dll
 0000:fffd0000       .debug$S                   0000000180000000     ucrt:api-ms-win-crt-string-l1-1-0.dll
 0000:fffd0000       .debug$S                   0000000180000000     ucrt:api-ms-win-crt-string-l1-1-0.dll
 0000:fffd0000       .debug$S                   0000000180000000     ucrt:api-ms-win-crt-string-l1-1-0.dll
 0000:fffd0000       .debug$S                   0000000180000000     ucrt:api-ms-win-crt-string-l1-1-0.dll
 0000:fffd0000       .debug$S                   0000000180000000     kernel32:KERNEL32.dll
 0000:fffd0000       .debug$S                   0000000180000000     kernel32:KERNEL32.dll
 0000:fffd0000       .debug$S                   0000000180000000     kernel32:KERNEL32.dll
 0000:fffd0000       .debug$S                   0000000180000000     kernel32:KERNEL32.dll
 0000:fffd0000       .debug$S                   0000000180000000     kernel32:KERNEL32.dll
 0000:fffd0000       .debug$S                   0000000180000000     kernel32:KERNEL32.dll
 0000:fffd0000       .debug$S                   0000000180000000     kernel32:KERNEL32.dll
 0000:fffd0000       .debug$S                   0000000180000000     kernel32:KERNEL32.dll
 0000:fffd0000       .debug$S                   0000000180000000     kernel32:KERNEL32.dll
 0000:fffd0000       .debug$S                   0000000180000000     kernel32:KERNEL32.dll
 0000:fffd0000       .debug$S                   0000000180000000     kernel32:KERNEL32.dll
 0000:fffd0000       .debug$S                   0000000180000000     kernel32:KERNEL32.dll
 0000:fffd0000       .debug$S                   0000000180000000     kernel32:KERNEL32.dll
 0000:fffd0000       .debug$S                   0000000180000000     kernel32:KERNEL32.dll
 0000:fffd0000       .debug$S                   0000000180000000     kernel32:KERNEL32.dll
 0000:fffd0000       .debug$S                   0000000180000000     kernel32:KERNEL32.dll
 0000:fffd0000       .debug$S                   0000000180000000     kernel32:KERNEL32.dll
 0000:fffd0000       .debug$S                   0000000180000000     kernel32:KERNEL32.dll
 0000:fffd0000       .debug$S                   0000000180000000     kernel32:KERNEL32.dll
 0000:fffd0000       .debug$S                   0000000180000000     kernel32:KERNEL32.dll
 0000:fffd0000       .debug$S                   0000000180000000     kernel32:KERNEL32.dll
 0000:fffd0000       .debug$S                   0000000180000000     kernel32:KERNEL32.dll
 0000:fffd0000       .debug$S                   0000000180000000     kernel32:KERNEL32.dll
 0000:fffd0000       .debug$S                   0000000180000000     kernel32:KERNEL32.dll
 0000:fffd0000       .debug$S                   0000000180000000     kernel32:KERNEL32.dll
 0000:fffd0000       .debug$S                   0000000180000000     kernel32:KERNEL32.dll
 0000:fffd0000       .debug$S                   0000000180000000     kernel32:KERNEL32.dll
 0000:fffd0000       .debug$S                   0000000180000000     kernel32:KERNEL32.dll
 0001:00000fe4       addRefToVerify             0000000180001fe4 f   libfollowref003.obj
 0001:00001050       agentProc                  0000000180002050 f   libfollowref003.obj
 0001:00001550       agentThreadWrapper         0000000180002550 f   libfollowref003.obj
 0001:000016f4       checkTestedObjects         00000001800026f4 f   libfollowref003.obj
 0001:00001890       check_option               0000000180002890 f   libfollowref003.obj
 0001:00001ad8       file_basename              0000000180002ad8 f   libfollowref003.obj
 0001:00001b4c       getChainObjects            0000000180002b4c f   libfollowref003.obj
 0001:00001db4       getTestedObjects           0000000180002db4 f   libfollowref003.obj
 0001:00003a80       registerFrame              0000000180004a80 f   libfollowref003.obj
 0001:00003b90       registerLocal              0000000180004b90 f   libfollowref003.obj
 0001:00003d44       registerThread             0000000180004d44 f   libfollowref003.obj
 0001:00003dd4       releaseTestedObjects       0000000180004dd4 f   libfollowref003.obj
 0001:00003f1c       setTagForTargetThread      0000000180004f1c f   libfollowref003.obj
 0001:00003fc8       startAgentThreadWrapper    0000000180004fc8 f   libfollowref003.obj
 0001:0000433c       syncDebuggeeStatus         000000018000533c f   libfollowref003.obj
 0001:000045dc       capture_previous_context   00000001800055dc f   MSVCRT:gs_report.obj
 0001:00004650       ?__scrt_initialize_thread_safe_statics@@YAHXZ 0000000180005650 f   MSVCRT:thread_safe_statics.obj
 0001:00004720       ?__scrt_uninitialize_thread_safe_statics@@YAXXZ 0000000180005720 f   MSVCRT:thread_safe_statics.obj
 0001:000047d0       $$000000                   00000001800057d0     MSVCRT:amdsecgs.obj
 0001:00004800       ?dllmain_crt_dispatch@@YAHQEAUHINSTANCE__@@KQEAX@Z 0000000180005800 f   MSVCRT:dll_dllmain.obj
 0001:00004850       ?dllmain_crt_process_attach@@YAHQEAUHINSTANCE__@@QEAX@Z 0000000180005850 f   MSVCRT:dll_dllmain.obj
 0001:00004968       ?dllmain_crt_process_detach@@YAH_N@Z 0000000180005968 f   MSVCRT:dll_dllmain.obj
 0001:000049ec       ?dllmain_dispatch@@YAHQEAUHINSTANCE__@@KQEAX@Z 00000001800059ec f   MSVCRT:dll_dllmain.obj
 0001:00005400       $$000000                   0000000180006400     MSVCRT:guard_dispatch.obj
 0001:00005420       $$000000                   0000000180006420     MSVCRT:guard_xfg_dispatch.obj
 0001:00005436       ?fin$0@?0??dllmain_crt_process_attach@@YAHQEAUHINSTANCE__@@QEAX@Z@4HA 0000000180006436 f   MSVCRT:dll_dllmain.obj
 0001:0000544d       ?fin$0@?0??dllmain_crt_process_detach@@YAH_N@Z@4HA 000000018000644d f   MSVCRT:dll_dllmain.obj
 0001:00005466       ?fin$1@?0??dllmain_crt_process_detach@@YAH_N@Z@4HA 0000000180006466 f   MSVCRT:dll_dllmain.obj
 0001:0000547a       ?filt$0@?0??dllmain_dispatch@@YAHQEAUHINSTANCE__@@KQEAX@Z@4HA 000000018000647a f   MSVCRT:dll_dllmain.obj
 0001:000054b0       __scrt_is_nonwritable_in_current_image$filt$0 00000001800064b0 f   MSVCRT:utility.obj
 0002:00000218       ?__scrt_initialize_tss_var@@3P6AHXZEA 0000000180007218     MSVCRT:thread_safe_statics.obj
 0002:00000340       ?opcLengths@@3QBEB         0000000180007340     libfollowref003.obj
 0002:000036d8       GS_ExceptionPointers       000000018000a6d8     MSVCRT:gs_report.obj
 0002:00003db0       $unwind$fprintf            000000018000adb0     libfollowref003.obj
 0002:00003dbc       $unwind$printf             000000018000adbc     libfollowref003.obj
 0002:00003dc8       $unwind$?NewObject@JNIEnv_@@QEAAPEAV_jobject@@PEAV_jclass@@PEAU_jmethodID@@ZZ 000000018000adc8     libfollowref003.obj
 0002:00003dc8       $unwind$nsk_lcomplain      000000018000adc8     libfollowref003.obj
 0002:00003dc8       $unwind$nsk_ldisplay       000000018000adc8     libfollowref003.obj
 0002:00003dd0       $unwind$nsk_jvmti_waitForSync 000000018000add0     libfollowref003.obj
 0002:00003dd0       $unwind$nsk_lvdisplay      000000018000add0     libfollowref003.obj
 0002:00003dd0       $unwind$_RTC_Initialize    000000018000add0     MSVCRT:initsect.obj
 0002:00003dd0       $unwind$_RTC_Terminate     000000018000add0     MSVCRT:initsect.obj
 0002:00003dd0       $unwind$?__scrt_initialize_thread_safe_statics@@YAHXZ 000000018000add0     MSVCRT:thread_safe_statics.obj
 0002:00003ddc       $unwind$nsk_complain       000000018000addc     libfollowref003.obj
 0002:00003ddc       $unwind$nsk_printf         000000018000addc     libfollowref003.obj
 0002:00003de4       $unwind$nsk_lvcomplain     000000018000ade4     libfollowref003.obj
 0002:00003dfc       $unwind$nsk_ltrace         000000018000adfc     libfollowref003.obj
 0002:00003dfc       $unwind$__report_gsfailure 000000018000adfc     MSVCRT:gs_report.obj
 0002:00003e04       $unwind$nsk_lvtrace        000000018000ae04     libfollowref003.obj
 0002:00003e04       $unwind$__raise_securityfailure 000000018000ae04     MSVCRT:gs_report.obj
 0002:00003e04       $unwind$__scrt_initialize_crt 000000018000ae04     MSVCRT:utility.obj
 0002:00003e04       $unwind$__scrt_initialize_onexit_tables 000000018000ae04     MSVCRT:utility.obj
 0002:00003e04       $unwind$__scrt_release_startup_lock 000000018000ae04     MSVCRT:utility.obj
 0002:00003e04       $unwind$__scrt_uninitialize_crt 000000018000ae04     MSVCRT:utility.obj
 0002:00003e04       $unwind$_onexit            000000018000ae04     MSVCRT:utility.obj
 0002:00003e0c       $unwind$nsk_lverify        000000018000ae0c     libfollowref003.obj
 0002:00003e1c       $unwind$nsk_vprintf        000000018000ae1c     libfollowref003.obj
 0002:00003e2c       $unwind$?nsk_jni_lverify@@YAHHPEAUJNIEnv_@@HQEBDH1ZZ 000000018000ae2c     libfollowref003.obj
 0002:00003e40       $unwind$?nsk_jni_check_exception@@YAHPEAUJNIEnv_@@QEBDH@Z 000000018000ae40     libfollowref003.obj
 0002:00003e5c       $unwind$nsk_jvmti_parseOptions 000000018000ae5c     libfollowref003.obj
 0002:00003e78       $unwind$nsk_jvmti_createJVMTIEnv 000000018000ae78     libfollowref003.obj
 0002:00003e8c       $unwind$Java_nsk_jvmti_unit_FollowReferences_FollowRefObjects_resetTags 000000018000ae8c     libfollowref003.obj
 0002:00003e8c       $unwind$addRefToVerify     000000018000ae8c     libfollowref003.obj
 0002:00003e8c       $unwind$nsk_jvmti_resetAgentData 000000018000ae8c     libfollowref003.obj
 0002:00003e8c       $unwind$nsk_jvmti_resumeSync 000000018000ae8c     libfollowref003.obj
 0002:00003e8c       $unwind$nsk_jvmti_setFailStatus 000000018000ae8c     libfollowref003.obj
 0002:00003e8c       $unwind$stringPrimitiveValueCallback 000000018000ae8c     libfollowref003.obj
 0002:00003e8c       $unwind$__scrt_initialize_default_local_stdio_options 000000018000ae8c     MSVCRT:default_local_stdio_options.obj
 0002:00003e8c       $unwind$?dllmain_crt_dispatch@@YAHQEAUHINSTANCE__@@KQEAX@Z 000000018000ae8c     MSVCRT:dll_dllmain.obj
 0002:00003e8c       $unwind$DllMain            000000018000ae8c     MSVCRT:dll_dllmain_stub.obj
 0002:00003e8c       $unwind$__GSHandlerCheck   000000018000ae8c     MSVCRT:gshandler.obj
 0002:00003e8c       $unwind$?__scrt_uninitialize_thread_safe_statics@@YAXXZ 000000018000ae8c     MSVCRT:thread_safe_statics.obj
 0002:00003e8c       $unwind$__scrt_acquire_startup_lock 000000018000ae8c     MSVCRT:utility.obj
 0002:00003e8c       $unwind$__scrt_dllmain_after_initialize_c 000000018000ae8c     MSVCRT:utility.obj
 0002:00003e8c       $unwind$__scrt_dllmain_before_initialize_c 000000018000ae8c     MSVCRT:utility.obj
 0002:00003e8c       $unwind$__scrt_dllmain_crt_thread_attach 000000018000ae8c     MSVCRT:utility.obj
 0002:00003e8c       $unwind$__scrt_dllmain_crt_thread_detach 000000018000ae8c     MSVCRT:utility.obj
 0002:00003e8c       $unwind$__scrt_dllmain_uninitialize_c 000000018000ae8c     MSVCRT:utility.obj
 0002:00003e8c       $unwind$__scrt_dllmain_uninitialize_critical 000000018000ae8c     MSVCRT:utility.obj
 0002:00003e8c       $unwind$atexit             000000018000ae8c     MSVCRT:utility.obj
 0002:00003e94       $unwind$check_option       000000018000ae94     libfollowref003.obj
 0002:00003e94       $unwind$nsk_jvmti_findOptionValue 000000018000ae94     libfollowref003.obj
 0002:00003e94       $unwind$_DllMainCRTStartup 000000018000ae94     MSVCRT:dll_dllmain.obj
 0002:00003ea4       $unwind$nsk_jvmti_findOptionIntValue 000000018000aea4     libfollowref003.obj
 0002:00003eb4       $unwind$nsk_jvmti_lverify  000000018000aeb4     libfollowref003.obj
 0002:00003ec8       $unwind$exitOnError        000000018000aec8     libfollowref003.obj
 0002:00003ed8       $unwind$Java_nsk_share_jvmti_ArgumentHandler_getAgentOptionsString 000000018000aed8     libfollowref003.obj
 0002:00003eec       $unwind$Java_nsk_jvmti_unit_FollowReferences_FollowRefObjects_getTag 000000018000aeec     libfollowref003.obj
 0002:00003eec       $unwind$Java_nsk_share_jvmti_DebugeeClass_checkStatus 000000018000aeec     libfollowref003.obj
 0002:00003eec       $unwind$agentThreadWrapper 000000018000aeec     libfollowref003.obj
 0002:00003efc       $unwind$startAgentThreadWrapper 000000018000aefc     libfollowref003.obj
 0002:00003f18       $unwind$registerFrame      000000018000af18     libfollowref003.obj
 0002:00003f18       $unwind$syncDebuggeeStatus 000000018000af18     libfollowref003.obj
 0002:00003f18       $unwind$__scrt_dllmain_exception_filter 000000018000af18     MSVCRT:utility.obj
 0002:00003f2c       $unwind$Java_nsk_share_jvmti_DebugeeClass_resetAgentData 000000018000af2c     libfollowref003.obj
 0002:00003f34       $unwind$MA_checkStatus     000000018000af34     libfollowref003.obj
 0002:00003f48       $unwind$Java_nsk_jvmti_unit_FollowReferences_FollowRefObjects_setTag 000000018000af48     libfollowref003.obj
 0002:00003f60       $unwind$Java_nsk_jvmti_unit_FollowReferences_FollowRefObjects_addRefToVerify 000000018000af60     libfollowref003.obj
 0002:00003f7c       $unwind$Agent_Initialize   000000018000af7c     libfollowref003.obj
 0002:00003f98       $unwind$getChainObjects    000000018000af98     libfollowref003.obj
 0002:00003fb4       $unwind$getTestedObjects   000000018000afb4     libfollowref003.obj
 0002:00003fcc       $unwind$checkTestedObjects 000000018000afcc     libfollowref003.obj
 0002:00003fe0       $unwind$releaseTestedObjects 000000018000afe0     libfollowref003.obj
 0002:00003ff8       $unwind$arrayPrimitiveValueCallback 000000018000aff8     libfollowref003.obj
 0002:00003ff8       $unwind$primitiveFieldCallback 000000018000aff8     libfollowref003.obj
 0002:00003ff8       $unwind$registerThread     000000018000aff8     libfollowref003.obj
 0002:00004000       $unwind$registerLocal      000000018000b000     libfollowref003.obj
 0002:0000401c       $unwind$heapReferenceCallback 000000018000b01c     libfollowref003.obj
 0002:00004034       $unwind$setTagForTargetThread 000000018000b034     libfollowref003.obj
 0002:00004048       $unwind$agentProc          000000018000b048     libfollowref003.obj
 0002:00004060       $unwind$capture_previous_context 000000018000b060     MSVCRT:gs_report.obj
 0002:0000406c       $unwind$__GSHandlerCheckCommon 000000018000b06c     MSVCRT:gshandler.obj
 0002:00004078       $xdatasym                  000000018000b078     MSVCRT:amdsecgs.obj
 0002:0000407c       $unwind$?dllmain_crt_process_attach@@YAHQEAUHINSTANCE__@@QEAX@Z 000000018000b07c     MSVCRT:dll_dllmain.obj
 0002:000040b8       $unwind$?fin$0@?0??dllmain_crt_process_attach@@YAHQEAUHINSTANCE__@@QEAX@Z@4HA 000000018000b0b8     MSVCRT:dll_dllmain.obj
 0002:000040b8       $unwind$?fin$0@?0??dllmain_crt_process_detach@@YAH_N@Z@4HA 000000018000b0b8     MSVCRT:dll_dllmain.obj
 0002:000040b8       $unwind$?fin$1@?0??dllmain_crt_process_detach@@YAH_N@Z@4HA 000000018000b0b8     MSVCRT:dll_dllmain.obj
 0002:000040c0       $unwind$?dllmain_crt_process_detach@@YAH_N@Z 000000018000b0c0     MSVCRT:dll_dllmain.obj
 0002:00004114       $unwind$?dllmain_dispatch@@YAHQEAUHINSTANCE__@@KQEAX@Z 000000018000b114     MSVCRT:dll_dllmain.obj
 0002:0000413c       $unwind$?filt$0@?0??dllmain_dispatch@@YAHQEAUHINSTANCE__@@KQEAX@Z@4HA 000000018000b13c     MSVCRT:dll_dllmain.obj
 0002:00004144       $unwind$__scrt_is_nonwritable_in_current_image 000000018000b144     MSVCRT:utility.obj
 0002:00004164       $unwind$__scrt_is_nonwritable_in_current_image$filt$0 000000018000b164     MSVCRT:utility.obj
 0002:0000416c       $unwind$__scrt_fastfail    000000018000b16c     MSVCRT:utility_desktop.obj
 0002:0000417c       $unwind$__security_init_cookie 000000018000b17c     MSVCRT:gs_support.obj
 0002:00004188       $unwind$__isa_available_init 000000018000b188     MSVCRT:cpu_disp.obj
 0002:00004198       $xdatasym                  000000018000b198     MSVCRT:guard_dispatch.obj
 0002:000041a0       $xdatasym                  000000018000b1a0     MSVCRT:guard_xfg_dispatch.obj
 0002:000041b0       .edata                     000000018000b1b0     followref003.exp
 0002:000041d8       rgpv                       000000018000b1d8     followref003.exp
 0002:00004210       rgszName                   000000018000b210     followref003.exp
 0002:00004248       rgwOrd                     000000018000b248     followref003.exp
 0002:00004264       szName                     000000018000b264     followref003.exp
 0002:00004275       $N00001                    000000018000b275     followref003.exp
 0002:00004284       $N00002                    000000018000b284     followref003.exp
 0002:00004291       $N00003                    000000018000b291     followref003.exp
 0002:000042d6       $N00004                    000000018000b2d6     followref003.exp
 0002:00004313       $N00005                    000000018000b313     followref003.exp
 0002:0000435b       $N00006                    000000018000b35b     followref003.exp
 0002:0000439b       $N00007                    000000018000b39b     followref003.exp
 0002:000043d8       $N00008                    000000018000b3d8     followref003.exp
 0002:00004413       $N00009                    000000018000b413     followref003.exp
 0002:00004441       $N00010                    000000018000b441     followref003.exp
 0002:00004472       $N00011                    000000018000b472     followref003.exp
 0002:000044a1       $N00012                    000000018000b4a1     followref003.exp
 0002:000044d0       $N00013                    000000018000b4d0     followref003.exp
 0002:00004505       $N00014                    000000018000b505     followref003.exp
 0002:0000496a       .idata$6                   000000018000b96a     kernel32:KERNEL32.dll
 0002:000049ce       .idata$6                   000000018000b9ce     vcruntime:VCRUNTIME140.dll
 0002:00004b60       .idata$6                   000000018000bb60     ucrt:api-ms-win-crt-heap-l1-1-0.dll
 0002:00004b80       .idata$6                   000000018000bb80     ucrt:api-ms-win-crt-runtime-l1-1-0.dll
 0002:00004ba2       .idata$6                   000000018000bba2     ucrt:api-ms-win-crt-convert-l1-1-0.dll
 0002:00004bc4       .idata$6                   000000018000bbc4     ucrt:api-ms-win-crt-stdio-l1-1-0.dll
 0002:00004be4       .idata$6                   000000018000bbe4     ucrt:api-ms-win-crt-string-l1-1-0.dll
 0003:00000000       ?codeAttributeName@@3PEBDEB 000000018000c000     libfollowref003.obj
 0003:00000008       ?lineNumberAttributeName@@3PEBDEB 000000018000c008     libfollowref003.obj
 0003:00000010       ?localVarAttributeName@@3PEBDEB 000000018000c010     libfollowref003.obj
 0003:00000018       ?localVarTypeAttributeName@@3PEBDEB 000000018000c018     libfollowref003.obj
 0003:00000020       ?stackMapAttributeName@@3PEBDEB 000000018000c020     libfollowref003.obj
 0003:00000028       ?callBytes@@3PAEA          000000018000c028     libfollowref003.obj
 0003:0000002c       ?allocBytes@@3PAEA         000000018000c02c     libfollowref003.obj
 0003:00000030       info                       000000018000c030     libfollowref003.obj
 0003:00000034       first_followref            000000018000c034     libfollowref003.obj
 0003:00000038       rootClassTag               000000018000c038     libfollowref003.obj
 0003:00000040       chainClassTag              000000018000c040     libfollowref003.obj
 0003:00000048       thrObjectTag               000000018000c048     libfollowref003.obj
 0003:00000050       rootObjectTag              000000018000c050     libfollowref003.obj
 0003:00000058       chainObjectTag             000000018000c058     libfollowref003.obj
 0003:00000060       ref_kind_str               000000018000c060     libfollowref003.obj
 0003:00000140       ?target_thread_name@?1??getTargetThread@@9@4PEBDEB 000000018000c140     libfollowref003.obj
 0003:0001abe4       redefineAttempted          0000000180026be4     libfollowref003.obj
 0003:0001abe8       nsk_context                0000000180026be8     libfollowref003.obj
 0003:0001abf4       redefineSucceed            0000000180026bf4     libfollowref003.obj
 0003:0001abf8       agentFailed                0000000180026bf8     libfollowref003.obj
 0003:0001abfc       currentAgentStatus         0000000180026bfc     libfollowref003.obj
 0003:0001ac00       context                    0000000180026c00     libfollowref003.obj
 0003:0001acb8       agentThread                0000000180026cb8     libfollowref003.obj
 0003:0001acc0       agentThreadProc            0000000180026cc0     libfollowref003.obj
 0003:0001acc8       agentThreadArg             0000000180026cc8     libfollowref003.obj
 0003:0001acd0       agent_data                 0000000180026cd0     libfollowref003.obj
 0003:0001ace0       jvmti_env                  0000000180026ce0     libfollowref003.obj
 0003:0001ace8       jvm                        0000000180026ce8     libfollowref003.obj
 0003:0001acf0       jni_env                    0000000180026cf0     libfollowref003.obj
 0003:0001acf8       checkStatus_func           0000000180026cf8     libfollowref003.obj
 0003:0001ad00       ?codeAttributeIndex@@3GA   0000000180026d00     libfollowref003.obj
 0003:0001ad04       ?lineNumberAttributeIndex@@3GA 0000000180026d04     libfollowref003.obj
 0003:0001ad08       ?localVarAttributeIndex@@3GA 0000000180026d08     libfollowref003.obj
 0003:0001ad0c       ?localVarTypeAttributeIndex@@3GA 0000000180026d0c     libfollowref003.obj
 0003:0001ad10       ?stackMapAttributeIndex@@3GA 0000000180026d10     libfollowref003.obj
 0003:0001ad14       ?stackFrameOffset@@3GA     0000000180026d14     libfollowref003.obj
 0003:0001ad18       ?mode@@3HA                 0000000180026d18     libfollowref003.obj
 0003:0001ad1c       ?constantPoolSize@@3GA     0000000180026d1c     libfollowref003.obj
 0003:0001ad20       ?orig@@3PEBEEB             0000000180026d20     libfollowref003.obj
 0003:0001ad28       ?gen@@3PEAEEA              0000000180026d28     libfollowref003.obj
 0003:0001ad30       ?inputPos@@3PEAEEA         0000000180026d30     libfollowref003.obj
 0003:0001ad38       ?endPos@@3PEBEEB           0000000180026d38     libfollowref003.obj
 0003:0001ad40       ?genPos@@3PEAEEA           0000000180026d40     libfollowref003.obj
 0003:0001ad48       ?markPos@@3PEAEEA          0000000180026d48     libfollowref003.obj
 0003:0001ad50       ?constantPool@@3PEAPEADEA  0000000180026d50     libfollowref003.obj
 0003:0001ad58       ?constantPoolCount@@3GA    0000000180026d58     libfollowref003.obj
 0003:0001ad5c       ?zeroBytes@@3PAEA          0000000180026d5c     libfollowref003.obj
 0003:0001ad60       ?codeLength@@3IA           0000000180026d60     libfollowref003.obj
 0003:0001ad64       chainLength                0000000180026d64     libfollowref003.obj
 0003:0001ad68       ?map@@3PEAIEA              0000000180026d68     libfollowref003.obj
 0003:0001ad70       ?widening@@3PEACEA         0000000180026d70     libfollowref003.obj
 0003:0001ad78       timeout                    0000000180026d78     libfollowref003.obj
 0003:0001ad80       objectsCount               0000000180026d80     libfollowref003.obj
 0003:0001ad84       fakeUserData               0000000180026d84     libfollowref003.obj
 0003:0001ad88       userDataError              0000000180026d88     libfollowref003.obj
 0003:0001ad8c       curr_frame_id              0000000180026d8c     libfollowref003.obj
 0003:0001ad90       objectDescList             0000000180026d90     libfollowref003.obj
 0003:0001ad98       curr_local_idx             0000000180026d98     libfollowref003.obj
 0003:0001ada0       heapCallbacks              0000000180026da0     libfollowref003.obj
 0003:0001ae20       thrDesc                    0000000180026e20     libfollowref003.obj
 0003:0001ee20       frameDesc                  000000018002ae20     libfollowref003.obj
 0003:00020620       locDesc                    000000018002c620     libfollowref003.obj
 0003:000212b0       GS_ExceptionRecord         000000018002d2b0     MSVCRT:gs_report.obj
 0003:00021350       GS_ContextRecord           000000018002d350     MSVCRT:gs_report.obj
 0003:00021820       ?g_tss_cv@@3U_RTL_CONDITION_VARIABLE@@A 000000018002d820     MSVCRT:thread_safe_statics.obj
 0003:00021828       ?g_tss_event@@3PEAXEA      000000018002d828     MSVCRT:thread_safe_statics.obj
 0003:00021830       ?g_tss_mutex@@3U_RTL_CRITICAL_SECTION@@A 000000018002d830     MSVCRT:thread_safe_statics.obj
 0003:00021858       ?g_sleep_condition_variable_cs@@3P6AHPEAU_RTL_CONDITION_VARIABLE@@PEAU_RTL_CRITICAL_SECTION@@K@ZEA 000000018002d858     MSVCRT:thread_safe_statics.obj
 0003:00021860       ?g_wake_all_condition_variable@@3P6AXPEAU_RTL_CONDITION_VARIABLE@@@ZEA 000000018002d860     MSVCRT:thread_safe_statics.obj
 0003:0002186c       ?__proc_attached@@3HA      000000018002d86c     MSVCRT:dll_dllmain.obj
 0003:00021880       ?is_initialized_as_dll@@3_NA 000000018002d880     MSVCRT:utility.obj
 0003:00021881       ?module_local_atexit_table_initialized@@3_NA 000000018002d881     MSVCRT:utility.obj
 0003:00021888       ?module_local_atexit_table@@3U_onexit_table_t@@A 000000018002d888     MSVCRT:utility.obj
 0003:000218a0       ?module_local_at_quick_exit_table@@3U_onexit_table_t@@A 000000018002d8a0     MSVCRT:utility.obj
